:020000040000FA
:0408000098EF0BF072
:1008100003B275EF05F0F2B493EF05F09EB09BEFD5
:1008200005F09EB2A3EF05F0F2A81AEF04F0F2B2C1
:1008300023EF04F0F2B01FEF04F047EF0BF0F29655
:10084000F29047EF0BF0CD90F2929EA02DEF04F0C6
:100850000101533F2DEF04F0542BB2C1B6F1B3C1E7
:10086000B7F1B4C1B8F1B5C1B9F1AEC1B2F1AFC120
:10087000B3F1B0C1B4F1B1C1B5F1AAC1AEF1ABC130
:10088000AFF1ACC1B0F1ADC1B1F1A6C1AAF1A7C140
:10089000ABF1A8C1ACF1A9C1ADF1A2C1A6F1A3C150
:1008A000A7F1A4C1A8F1A5C1A9F19EC1A2F19FC160
:1008B000A3F1A0C1A4F1A1C1A5F19AC19EF19BC170
:1008C0009FF19CC1A0F19DC1A1F1CECF9AF1CFCFF4
:1008D0009BF153C19CF154C19DF1CF6ACE6A0101D5
:1008E000536B546B9E90CD800FBC0F8E0FBA7CEF74
:1008F00004F00F8A47EF0BF013880F8C0FBEB9EF8F
:1009000004F09AC19EF19BC19FF19CC1A0F19DC1D1
:10091000A1F19EC1A2F19FC1A3F1A0C1A4F1A1C107
:10092000A5F1A2C1A6F1A3C1A7F1A4C1A8F1A5C1D7
:10093000A9F1A6C1AAF1A7C1ABF1A8C1ACF1A9C1A7
:10094000ADF1AAC1AEF1ABC1AFF1ACC1B0F1ADC177
:10095000B1F1AEC1B2F1AFC1B3F1B0C1B4F1B1C147
:10096000B5F1B2C1B6F1B3C1B7F1B4C1B8F1B5C117
:10097000B9F101015E6B5F6B606B616B9A515E2731
:100980009B515F239C5160239D5161239E515E27A3
:100990009F515F23A0516023A1516123A2515E2783
:1009A000A3515F23A4516023A5516123A6515E2763
:1009B000A7515F23A8516023A9516123AA515E2743
:1009C000AB515F23AC516023AD516123AE515E2723
:1009D000AF515F23B0516023B1516123B2515E2703
:1009E000B3515F23B4516023B5516123B6515E27E3
:1009F000B7515F23B8516023B9516123D8900101E9
:100A0000613360335F335E33D8900101613360330B
:100A10005F335E33D8900101613360335F335E33FF
:100A200000C10CF101C10DF102C10EF103C10FF1C2
:100A300004C110F105C111F106C112F107C113F192
:100A400008C114F109C115F10AC116F10BC117F162
:100A500034C135F111B838EF05F00101620E046FB1
:100A6000010E056F000E066F000E076F41EF05F0D7
:100A70000101A70E046F020E056F000E066F000E37
:100A8000076F5EC100F15FC101F160C102F161C198
:100A900003F167EC2FF003BF04D01CBE02D01CA0F2
:100AA000108C11A059EF05F010BA59EF05F00F8026
:100AB000108A0CC100F10DC101F10EC102F10FC18C
:100AC00003F110C104F111C105F112C106F113C106
:100AD00007F114C108F115C109F116C10AF117C1D6
:100AE0000BF135C134F147EF0BF00392ABB2AB9889
:100AF000AB88030103EE00F080517F0BE92604C0B0
:100B0000EFFF802B8151805D700BD8A48B82000099
:100B10008051815D700BD8A48B9281518019D8B41B
:100B2000079047EF0BF0F2940101453F47EF0BF0C0
:100B3000462B47EF0BF09E900101533F47EF0BF020
:100B4000542B47EF0BF09E9211B843EF08F00400CE
:100B500066A1ABEF05F08BB4B5EF05F010ACB5EFC7
:100B600005F08B84109CB6EF05F08B94077C07ACE6
:100B7000D1EF05F0C274C2B4CBEF05F0C3CFB7F527
:100B8000C4CFB8F50501D890B833B733D890B8338F
:100B9000B733D2EF05F0C3CF55F1C4CF56F1D2EF42
:100BA00005F0C28207B444EF06F047C14BF148C1DB
:100BB0004CF149C14DF14AC14EF15EC162F15FC1D4
:100BC00063F160C164F161C165F113A8EAEF05F05A
:100BD000138C13989AC1BAF19BC1BBF19CC1BCF1B3
:100BE0009DC1BDF19EC1BEF19FC1BFF1A0C1C0F1C9
:100BF000A1C1C1F1A2C1C2F1A3C1C3F1A4C1C4F199
:100C0000A5C1C5F1A6C1C6F1A7C1C7F1A8C1C8F168
:100C1000A9C1C9F1AAC1CAF1ABC1CBF1ACC1CCF138
:100C2000ADC1CDF1AEC1CEF1AFC1CFF1B0C1D0F108
:100C3000B1C1D1F1B2C1D2F1B3C1D3F1B4C1D4F1D8
:100C4000B5C1D5F1B6C1D6F1B7C1D7F1B8C1D8F1A8
:100C5000B9C1D9F1B7C5B9F5B8C5BAF5B9C5BBF5CC
:100C6000BAC5BCF5010155515B2756515C23E86AB2
:100C70005D230E2E44EF06F05CC157F15DC158F1C3
:100C80005B6B5C6B5D6B078E0201002F47EF0BF017
:100C90003C0E006F1D50E00BE00AE86612881BBE98
:100CA00002D01BB4108E00C10CF101C10DF102C1C4
:100CB0000EF103C10FF104C110F105C111F106C11C
:100CC00012F107C113F108C114F109C115F10AC1EC
:100CD00016F10BC117F134C135F181AAACEF06F062
:100CE00015A4F7EF06F005012F51000AD8B43AEF2A
:100CF00007F005012F51010AD8B4B6EF06F005013F
:100D00002F51020AD8B4F7EF06F005012F51030A5C
:100D1000D8B4F7EF06F005012F51040AD8B4F7EF65
:100D200006F005012F51050AD8B4F7EF06F00501CA
:100D30002F51060AD8B4F7EF06F005012F51070A24
:100D4000D8B4F7EF06F005012F51320AD8B4B4EF4A
:100D500006F02F6B3AEF07F000011650030AD8B4E3
:100D6000F7EF06F03AEF07F03AEF07F005015767A3
:100D7000C1EF06F05867C1EF06F05967C1EF06F002
:100D80005A67C5EF06F03AEF07F05BC500F15CC5A6
:100D900001F15DC502F15EC503F10101010E046FB1
:100DA000000E056F000E066F000E076F67EC2FF048
:100DB00000C15BF501C15CF502C15DF503C15EF5E3
:100DC00001010067EBEF06F00167EBEF06F0026749
:100DD000EBEF06F003673AEF07F057C55BF558C530
:100DE0005CF559C55DF55AC55EF524EF07F00FBEF9
:100DF0000CEF07F010A011EF07F00101476708EFB3
:100E000007F0486708EF07F0496708EF07F04A67FF
:100E10000CEF07F011EF07F007AE11EF07F024EF2A
:100E200007F00501312F3AEF07F03C0E316F302FFC
:100E30003AEF07F00101000E626FE00E636FA50E3E
:100E4000646F010E656F138800011650000AD8B454
:100E500032EF07F000011650030AD8B437EF07F05D
:100E60003AEF07F00001010E166E3AEF07F00001AD
:100E7000040E166E0501666B37B740EF07F066810A
:100E80000CC100F10DC101F10EC102F10FC103F15E
:100E900010C104F111C105F112C106F113C107F12E
:100EA00014C108F115C109F116C10AF117C10BF1FE
:100EB00035C134F100C10CF101C10DF102C10EF1D7
:100EC00003C10FF104C110F105C111F106C112F106
:100ED00007C113F108C114F109C115F10AC116F1D6
:100EE0000BC117F134C135F101018E677FEF07F0B7
:100EF0008F677FEF07F090677FEF07F0916783EFD1
:100F000007F0B4EF07F092C100F193C101F194C171
:100F100002F195C103F10101010E046F000E056F8E
:100F2000000E066F000E076F67EC2FF000C192F104
:100F300001C193F102C194F103C195F10101006770
:100F4000A9EF07F00167A9EF07F00267A9EF07F023
:100F50000367B4EF07F08EC192F18FC193F190C196
:100F600094F191C195F10F80D57ED5BE6ED0D6CFCC
:100F700047F1D7CF48F145C149F1E86AE8CF4AF1D6
:100F8000138A1CBE02D01CA0108C109047C100F127
:100F900048C101F149C102F14AC103F101010A0E40
:100FA000046F000E056F000E066F000E076F67ECF2
:100FB0002FF003AF1080010154A7EBEF07F00F9A59
:100FC0000F9C0F9E0101000E5E6F600E5F6F3D0E65
:100FD000606F080E616F010147BFFBEF07F04867C4
:100FE000FBEF07F04967FBEF07F04A67FBEF07F0FD
:100FF000F28820EF08F0F2985E6B5F6B606B616BBC
:101000009A6B9B6B9C6B9D6B9E6B9F6BA06BA16B9C
:10101000A26BA36BA46BA56BA66BA76BA86BA96B4C
:10102000AA6BAB6BAC6BAD6BAE6BAF6BB06BB16BFC
:10103000B26BB36BB46BB56BB66BB76BB86BB96BAC
:10104000D76AD66A0101456B466B0CC100F10DC130
:1010500001F10EC102F10FC103F110C104F111C180
:1010600005F112C106F113C107F114C108F115C150
:1010700009F116C10AF117C10BF135C134F147EF7F
:101080000BF047EF0BF00201002FABEF0AF0D59EFB
:10109000D6CF47F1D7CF48F145C149F1E86AE8CF4B
:1010A0004AF1138AD76AD66A0101456B466BD58E21
:1010B0001D50E00BE00AE86612881BBE02D01BB48C
:1010C000108E1AAE1F8C00C10CF101C10DF102C1CE
:1010D0000EF103C10FF104C110F105C111F106C1F8
:1010E00012F107C113F108C114F109C115F10AC1C8
:1010F00016F10BC117F134C135F10FA0109A11B8D8
:101100008DEF08F00101620E046F010E056F000EF5
:10111000066F000E076F96EF08F00101A70E046F2F
:10112000020E056F000E066F000E076F47C100F13B
:1011300048C101F149C102F14AC103F167EC2FF046
:1011400003BFA9EF08F01CBE02D01CA0108C11B088
:101150000F800CC100F10DC101F10EC102F10FC1F0
:1011600003F110C104F111C105F112C106F113C15F
:1011700007F114C108F115C109F116C10AF117C12F
:101180000BF135C134F102013C0E006F00C10CF1CE
:1011900001C10DF102C10EF103C10FF104C110F143
:1011A00005C111F106C112F107C113F108C114F113
:1011B00009C115F10AC116F10BC117F134C135F19E
:1011C00081BAE6EF08F015B225EF09F015A025EF7A
:1011D00009F015A470EF09F005012F51000AD8B4E9
:1011E000B3EF09F005012F51010AD8B42FEF09F030
:1011F00005012F51020AD8B470EF09F005012F51F3
:10120000030AD8B470EF09F005012F51040AD8B4CD
:1012100070EF09F005012F51050AD8B470EF09F0FD
:1012200005012F51060AD8B470EF09F005012F51BE
:10123000070AD8B470EF09F005012F51320AD8B46B
:101240002DEF09F02F6BB3EF09F000011650030AE0
:10125000D8B470EF09F0B3EF09F0B3EF09F005016E
:1012600057673AEF09F058673AEF09F059673AEFD4
:1012700009F05A673EEF09F0B3EF09F05BC500F1E2
:101280005CC501F15DC502F15EC503F10101010E0E
:10129000046F000E056F000E066F000E076F67ECFF
:1012A0002FF000C15BF501C15CF502C15DF503C122
:1012B0005EF50101006764EF09F0016764EF09F072
:1012C000026764EF09F00367B3EF09F057C55BF5F8
:1012D00058C55CF559C55DF55AC55EF59DEF09F039
:1012E0000FBE85EF09F010A08AEF09F001014767F2
:1012F00081EF09F0486781EF09F0496781EF09F054
:101300004A6785EF09F08AEF09F007AE8AEF09F026
:101310009DEF09F00501312FB3EF09F03C0E316F5D
:10132000302FB3EF09F00101000E626FE00E636F22
:10133000A50E646F010E656F138800011650000A38
:10134000D8B4ABEF09F000011650030AD8B4B0EFDF
:1013500009F0B3EF09F00001010E166EB3EF09F0CA
:101360000001040E166E0501666B37B7B9EF09F080
:1013700066810CC100F10DC101F10EC102F10FC176
:1013800003F110C104F111C105F112C106F113C13D
:1013900007F114C108F115C109F116C10AF117C10D
:1013A0000BF135C134F100C10CF101C10DF102C1E5
:1013B0000EF103C10FF104C110F105C111F106C115
:1013C00012F107C113F108C114F109C115F10AC1E5
:1013D00016F10BC117F134C135F101018E67F8EF39
:1013E00009F08F67F8EF09F09067F8EF09F091675F
:1013F000FCEF09F02DEF0AF092C100F193C101F169
:1014000094C102F195C103F10101010E046F000EB8
:10141000056F000E066F000E076F67EC2FF000C11E
:1014200092F101C193F102C194F103C195F101015F
:10143000006722EF0AF0016722EF0AF0026722EF4D
:101440000AF003672DEF0AF08EC192F18FC193F17C
:1014500090C194F191C195F10F80109047C100F1B6
:1014600048C101F149C102F14AC103F101010A0E6B
:10147000046F000E056F000E066F000E076F67EC1D
:101480002FF003AF1080010154A753EF0AF00F9A19
:101490000F9C0F9E0101000E5E6F600E5F6F3D0E90
:1014A000606F080E616F47C100F148C101F149C189
:1014B00002F14AC103F10101140E046F050E056F1C
:1014C000000E066F000E076F67EC2FF003AF6CEF96
:1014D0000AF0F28891EF0AF0F2985E6B5F6B606B36
:1014E000616B9A6B9B6B9C6B9D6B9E6B9F6BA06BF8
:1014F000A16BA26BA36BA46BA56BA66BA76BA86B70
:10150000A96BAA6BAB6BAC6BAD6BAE6BAF6BB06B1F
:10151000B16BB26BB36BB46BB56BB66BB76BB86BCF
:10152000B96B0CC100F10DC101F10EC102F10FC187
:1015300003F110C104F111C105F112C106F113C18B
:1015400007F114C108F115C109F116C10AF117C15B
:101550000BF135C134F104008BB4B6EF0AF010ACD6
:10156000B6EF0AF08B84109CB7EF0AF08B94077CDF
:1015700007ACD2EF0AF0C274C2B4CCEF0AF0C3CF0A
:10158000B7F5C4CFB8F50501D890B833B733D890C4
:10159000B833B733D3EF0AF0C3CF55F1C4CF56F108
:1015A000D3EF0AF0C28207B445EF0BF047C14BF10D
:1015B00048C14CF149C14DF14AC14EF15EC162F1E1
:1015C0005FC163F160C164F161C165F113A8EBEF24
:1015D0000AF0138C13989AC1BAF19BC1BBF19CC15C
:1015E000BCF19DC1BDF19EC1BEF19FC1BFF1A0C1C3
:1015F000C0F1A1C1C1F1A2C1C2F1A3C1C3F1A4C193
:10160000C4F1A5C1C5F1A6C1C6F1A7C1C7F1A8C162
:10161000C8F1A9C1C9F1AAC1CAF1ABC1CBF1ACC132
:10162000CCF1ADC1CDF1AEC1CEF1AFC1CFF1B0C102
:10163000D0F1B1C1D1F1B2C1D2F1B3C1D3F1B4C1D2
:10164000D4F1B5C1D5F1B6C1D6F1B7C1D7F1B8C1A2
:10165000D8F1B9C1D9F1B7C5B9F5B8C5BAF5B9C5A9
:10166000BBF5BAC5BCF5010155515B2756515C234A
:10167000E86A5D230E2E45EF0BF05CC157F15DC1AA
:1016800058F15B6B5C6B5D6B078E47EF0BF002C034
:10169000E0FF005001C0D8FF1000A6B24DEF0BF0E4
:1016A0000CC0A9FF0BC0A8FFA69EA69CA684F29E14
:1016B000550EA76EAA0EA76EA682F28EA694A6B2AB
:1016C0005FEF0BF00C2A1200A96EA69EA69CA680C6
:1016D000A8500C2A120004012C0E826F94EC0EF01C
:1016E00062EC30F00C5064EC0BF0E8CF00F10C50E1
:1016F00064EC0BF0E8CF01F101AF84EF0BF00101D6
:10170000FF0E026FFF0E036F05EC30F0296790EFBC
:101710000BF00401200E826F94EC0EF095EF0BF0AD
:1017200004012D0E826F94EC0EF00FEC2EF01200DF
:1017300015941596076A0F6A106A116A126A136A7D
:10174000166A0F010D0EC16E860EC06E030EC26EBC
:101750000F01680E896E130E926E080E8A6EF30EDC
:10176000936E8B6A900E946EC80E64EC0BF0E8CF0B
:10177000E8FF1098E8A0108810A805D00E0E256E7E
:101780008E0E266E04D00F0E256E8F0E266EFAEC8E
:1017900030F0F18EF19EFC0E64EC0BF0E8CF0BF014
:1017A0000BA011800BA211820BA411840BA811882D
:1017B000C90E64EC0BF0E8CF1AF0CA0E64EC0BF023
:1017C000E8CF1BF0CB0E64EC0BF0E8CF1CF0CC0E96
:1017D00064EC0BF0E8CF1DF0FB0E64EC0BF0E8CFEF
:1017E00037F0CE0E64EC0BF0E8CF14F0CD0E64ECC5
:1017F0000BF0E8CF36F01F6A206A0E6A01015B6BBE
:101800005C6B5D6B576B586BF29A0101476B486BD1
:10181000496B4A6B4B6B4C6B4D6B4E6B4F6B506B0C
:10182000516B526B456B466BD76AD66A0F01280E17
:10183000D56EF28A9D90B00ECD6E01015E6B5F6B2E
:10184000606B616B626B636B646B656B666B676B24
:10185000686B696B536B546BCF6ACE6A0F9A0F9C9F
:101860000F9E9D80760ECA6E9D8202013C0E006F17
:10187000CC6A160E64EC0BF0E8CF00F1170E64ECA6
:101880000BF0E8CF01F1180E64EC0BF0E8CF02F199
:10189000190E64EC0BF0E8CF03F1010103AF6BEF1D
:1018A0000CF062EC30F0160E0C6E00C10BF04DEC3B
:1018B0000BF0170E0C6E01C10BF04DEC0BF0180E77
:1018C0000C6E02C10BF04DEC0BF0190E0C6E03C147
:1018D0000BF04DEC0BF000C18EF101C18FF102C194
:1018E00090F103C191F100C192F101C193F102C1E4
:1018F00094F103C195F11A0E64EC0BF0E8CF00F1FE
:101900001B0E64EC0BF0E8CF01F11C0E64EC0BF045
:10191000E8CF02F11D0E64EC0BF0E8CF03F10101FA
:1019200003AFC1EF0CF062EC30F01A0E0C6E00C188
:101930000BF04DEC0BF01B0E0C6E01C10BF04DECDF
:101940000BF01C0E0C6E02C10BF04DEC0BF01D0EDB
:101950000C6E03C10BF04DEC0BF01A0E64EC0BF0A7
:10196000E8CF00F11B0E64EC0BF0E8CF01F11C0E88
:1019700064EC0BF0E8CF02F11D0E64EC0BF0E8CF45
:1019800003F100C196F101C197F102C198F103C1C1
:1019900099F1240EAC6E900EAB6E240EAC6E080E58
:1019A000B86E000EB06E1F0EAF6E0401806B816BBF
:1019B0000F01900EAB6E0F019D8A0301806B816B4E
:1019C000C26B8B929FEC35F09FEC35F05AEC37F000
:1019D0007DEC33F0200E64EC0BF0E8CF2FF5050121
:1019E0002F51FF0AD8A4FCEF0CF02F6B200E0C6EC9
:1019F0002FC50BF04DEC0BF00501010E306F3C0EC6
:101A0000316F250E64EC0BF0E8CF00F1260E64EC8C
:101A10000BF0E8CF01F1270E64EC0BF0E8CF02F1F8
:101A2000280E64EC0BF0E8CF03F1010103AF33EFB4
:101A30000DF062EC30F0250E0C6E00C10BF04DEC99
:101A40000BF0260E0C6E01C10BF04DEC0BF0270EC7
:101A50000C6E02C10BF04DEC0BF0280E0C6E03C1A6
:101A60000BF04DEC0BF000C157F501C158F502C168
:101A700059F503C15AF500C15BF501C15CF502C11E
:101A80005DF503C15EF5290E64EC0BF0E8CF5FF560
:101A9000050160515F5DD8A05FC560F5210E64EC63
:101AA0000BF0E8CF00F1220E64EC0BF0E8CF01F16F
:101AB000230E64EC0BF0E8CF02F1240E64EC0BF083
:101AC000E8CF03F1010103AF94EF0DF062EC30F0C9
:101AD000210E0C6E00C10BF04DEC0BF0220E0C6EC3
:101AE00001C10BF04DEC0BF0230E0C6E02C10BF09C
:101AF0004DEC0BF0240E0C6E03C10BF04DEC0BF013
:101B0000210E64EC0BF0E8CF00F1220E64EC0BF038
:101B1000E8CF01F1230E64EC0BF0E8CF02F1240EC4
:101B200064EC0BF0E8CF03F100C161F501C162F58F
:101B300002C163F503C164F5C5EC32F0ABEC31F0E2
:101B400003EC31F01590C70E64EC0BF0E8CF00F118
:101B5000010100B1AFEF0DF01592B0EF0DF015825D
:101B600081AABEEF0DF015B4B9EF0DF01580BEEFF0
:101B70000DF099EC37F015A0FCEF37F0079000015D
:101B8000F28EF28C12AE03D012BC6CEF19F007B0DB
:101B90009CEF2CF00FB098EF25F010BE98EF25F0D9
:101BA00012B898EF25F000011650010AD8B49FEF43
:101BB0001DF081BAE4EF0DF000011650040AD8B40C
:101BC00018EF1CF0EAEF0DF000011650040AD8B42B
:101BD000D4EF1DF00301805181197F0BD8B49CEF25
:101BE0002CF013EE00F081517F0BE126812BE7CF23
:101BF000E8FFE00BD8B49CEF2CF023EE82F0C2514A
:101C00003F0BD926E7CFDFFFC22BDF50780AD8A4DD
:101C10009CEF2CF0078092C100F193C101F194C1B7
:101C200002F195C103F10101040E046F000E056F6E
:101C3000000E066F000E076F67EC2FF000AF2AEF63
:101C40000EF00101030E926F000E936F000E946F61
:101C5000000E956F03018251720AD8B419EF25F076
:101C60008251520AD8B419EF25F08251750AD8B4BE
:101C700019EF25F08251680AD8B4A8EF0EF082510E
:101C8000630AD8B456EF29F08251690AD8B4D7EF65
:101C900020F082517A0AD8B4EAEF21F08251490A41
:101CA000D8B476EF20F08251500AD8B494EF1FF0E8
:101CB0008251700AD8B4D7EF1FF08251540AD8B4B9
:101CC00002EF20F08251740AD8B448EF20F082511C
:101CD000410AD8B4ADEF0FF082514B0AD8B4AAEF45
:101CE0000EF082516D0AD8B41DEF14F082514D0AE6
:101CF000D8B436EF14F08251730AD8B449EF24F007
:101D00008251530AD8B4AEEF24F082514C0AD8B4B1
:101D1000C5EF14F08251590AD8B46EEF13F012AE29
:101D200001D0128C8DEF29F0040114EE00F08051E7
:101D30007F0BE12682C4E7FF802B120004010D0E09
:101D4000826F94EC0EF00A0E826F94EC0EF012008B
:101D50008BEF29F004014B0E826F94EC0EF004011E
:101D60002C0E826F94EC0EF081B802D036B630D0D3
:101D700003018351430AD8B4EFEF0EF003018351FE
:101D8000630AD8B4F1EF0EF003018351520AD8B4BC
:101D9000F3EF0EF003018351720AD8B4F5EF0EF0A1
:101DA00003018351470AD8B4F7EF0EF003018351C2
:101DB000670AD8B4F9EF0EF003018351540AD8B47E
:101DC000FBEF0EF003018351740AD8B46BEF0FF0F0
:101DD00003018351550AD8B4FDEF0EF083D036804D
:101DE0007BD0369079D0368277D0369275D03684D3
:101DF00073D0369471D036866FD084C330F185C3EA
:101E000031F186C332F187C333F10101296BB0ECA4
:101E100030F027EC30F000C104F101C105F102C13E
:101E200006F103C107F1A3EC30F0200EF86EF76A5B
:101E3000F66A0900F5CF2CF10900F5CF2DF1090064
:101E4000F5CF2EF10900F5CF2FF10900F5CF30F1D4
:101E50000900F5CF31F10900F5CF32F10900F5CFD6
:101E600033F10101296BB0EC30F027EC30F067EC76
:101E70002FF00101006744EF0FF0016744EF0FF00E
:101E8000026744EF0FF0036701D025D004014E0E26
:101E9000826F94EC0EF004016F0E826F94EC0EF0E2
:101EA00004014D0E826F94EC0EF00401610E826FFE
:101EB00094EC0EF00401740E826F94EC0EF00401A9
:101EC000630E826F94EC0EF00401680E826F94EC46
:101ED0000EF08BEF29F03696CD0E0C6E36C00BF05F
:101EE0004DEC0BF0CD0E64EC0BF0E8CF36F036B0D5
:101EF00006D00401630E826F94EC0EF005D004014D
:101F0000430E826F94EC0EF036B206D00401720ECE
:101F1000826F94EC0EF005D00401520E826F94ECA7
:101F20000EF036B406D00401670E826F94EC0EF00A
:101F300005D00401470E826F94EC0EF036B606D041
:101F40000401740E826F94EC0EF005D00401540E5F
:101F5000826F94EC0EF08BEF29F00401410E826F3A
:101F600094EC0EF003018351310AD8B48EEF12F0D5
:101F700003018351320AD8B4BEEF11F0030183513B
:101F8000330AD8B447EF11F003018351340AD8B4AF
:101F900037EF10F003018351350AD8B4D7EF0FF0B3
:101FA00004013F0E826F94EC0EF08BEF29F00301D9
:101FB0008451300AD8B4FDEF0FF003018451310A87
:101FC000D8B400EF10F003018451650AD8B4F1EFE2
:101FD0000FF003018451640AD8B4F4EF0FF001EF5D
:101FE00010F03790F5EF0FF03780FB0E0C6E37C016
:101FF0000BF04DEC0BF001EF10F08B9001EF10F0B7
:102000008B800401350E826F94EC0EF004012C0ECF
:10201000826F94EC0EF08BB015EF10F00401300ECF
:10202000826F94EC0EF01AEF10F00401310E826F03
:1020300094EC0EF004012C0E826F94EC0EF0FB0E6B
:1020400064EC0BF0E8CF37F037A02EEF10F004016E
:10205000640E826F94EC0EF033EF10F00401650E05
:10206000826F94EC0EF035EF10F08BEF29F0CC0E70
:1020700064EC0BF0E8CF0BF004012C0E826F94ECB3
:102080000EF003018451310AD8B45BEF10F0030164
:102090008451300AD8B45DEF10F0030184514D0A29
:1020A000D8B467EF10F003018451540AD8B46EEF2E
:1020B00010F085EF10F08A8401D08A940BAE04D022
:1020C0000BAC02D00BBA21D0E00E0B1218D01F0EB1
:1020D0000B168539E844E00B0B1211D0E00E0B16FD
:1020E000A3EC30F085C332F186C333F10101296BD3
:1020F000B0EC30F027EC30F000511F0B0B12CC0E7F
:102100000C6E0BC00BF04DEC0BF00401340E826F23
:1021100094EC0EF004012C0E826F94EC0EF0CC0EB9
:1021200064EC0BF0E8CF1DF08AB406D00401300E49
:10213000826F94EC0EF005D00401310E826F94ECA6
:102140000EF004012C0E826F94EC0EF01D38E84066
:10215000070BE8CF82F40401300E822794EC0EF0D6
:1021600004012C0E826F94EC0EF062EC30F01D50E6
:102170001F0BE8CF00F105EC30F032C182F404010E
:10218000300E822794EC0EF033C182F40401300E3D
:10219000822794EC0EF004012C0E826F94EC0EF06A
:1021A00062EC30F030C000F100AF0BD0FF0E016FD9
:1021B000FF0E026FFF0E036F04012D0E826F94EC71
:1021C0000EF005EC30F031C182F40401300E8227AC
:1021D00094EC0EF032C182F40401300E822794ECAC
:1021E0000EF033C182F40401300E822794EC0EF01D
:1021F00004012C0E826F94EC0EF062EC30F02FC0D4
:1022000000F105EC30F031C182F40401300E822778
:1022100094EC0EF032C182F40401300E822794EC6B
:102220000EF033C182F40401300E822794EC0EF0DC
:1022300004012C0E826F94EC0EF062EC30F031C091
:1022400000F100AF0BD0FF0E016FFF0E026FFF0E0B
:10225000036F04012D0E826F94EC0EF005EC30F04C
:1022600031C182F40401300E822794EC0EF032C1A9
:1022700082F40401300E822794EC0EF033C182F414
:102280000401300E822794EC0EF08BEF29F0CB0E78
:1022900064EC0BF0E8CF0BF004012C0E826F94EC91
:1022A0000EF003018451450AD8B46BEF11F003011D
:1022B0008451440AD8B46EEF11F003018451300AFE
:1022C000D8B471EF11F003018451310AD8B475EF1D
:1022D00011F080EF11F00B9E7AEF11F00B8E7AEF78
:1022E00011F0FC0E0B167AEF11F0FC0E0B160B80A2
:1022F0007AEF11F0CB0E0C6E0BC00BF04DEC0BF027
:102300000401330E826F94EC0EF004012C0E826FE8
:1023100094EC0EF0CB0E64EC0BF0E8CF1CF01CBE7E
:1023200099EF11F00401450E826F94EC0EF09EEFD0
:1023300011F00401440E826F94EC0EF004012C0E97
:10234000826F94EC0EF00401300E826F94EC0EF06C
:1023500004012C0E826F94EC0EF01CB0B7EF11F05C
:102360000401300E826F94EC0EF0BCEF11F004010A
:10237000310E826F94EC0EF08BEF29F0CA0E64ECF4
:102380000BF0E8CF0BF004012C0E826F94EC0EF0F2
:1023900003018451450AD8B4FAEF11F003018451C6
:1023A000440AD8B4FDEF11F0030184514D0AD8B4AA
:1023B00006EF12F003018451410AD8B400EF12F085
:1023C00003018451460AD8B403EF12F0030184518B
:1023D000560AD8B40EEF12F003018451500AD8B453
:1023E00019EF12F003018451520AD8B41CEF12F015
:1023F00025EF12F00B9E1FEF12F00B8E1FEF12F065
:102400000B9C1FEF12F00B8C1FEF12F0FC0E0B1643
:1024100085C3E8FF030B0B121FEF12F0C70E0B165C
:1024200085C3E8FF070BE846E846E8460B121FEFB6
:1024300012F00B841FEF12F00B941FEF12F0CA0E74
:102440000C6E0BC00BF04DEC0BF0CA0E64EC0BF0F5
:10245000E8CF1BF00401320E826F94EC0EF0040101
:102460002C0E826F94EC0EF01BBE3EEF12F00401B6
:10247000450E826F94EC0EF043EF12F00401440E0F
:10248000826F94EC0EF004012C0E826F94EC0EF02F
:102490001BC0E8FF030BE8CF82F40401300E822753
:1024A00094EC0EF004012C0E826F94EC0EF01BBC29
:1024B00061EF12F00401410E826F94EC0EF066EFB2
:1024C00012F00401460E826F94EC0EF004012C0E03
:1024D000826F94EC0EF01BC0E8FF380BE842E84234
:1024E000E842E8CF82F40401300E822794EC0EF02B
:1024F00004012C0E826F94EC0EF01BB487EF12F0E7
:102500000401520E826F94EC0EF08CEF12F0040175
:10251000500E826F94EC0EF08BEF29F0C90E64EC34
:102520000BF0E8CF0BF004012C0E826F94EC0EF050
:1025300003018451450AD8B4ACEF12F00301845171
:10254000440AD8B4AFEF12F0030184514D0AD8B455
:10255000B2EF12F0C0EF12F00B9EBAEF12F00B8E3A
:10256000BAEF12F0F80E0B1685C3E8FF070B0B123B
:10257000BAEF12F0C90E0C6E0BC00BF04DEC0BF065
:102580000401310E826F94EC0EF004012C0E826F68
:1025900094EC0EF0C90E64EC0BF0E8CF1AF01ABE02
:1025A00006D00401450E826F94EC0EF005D00401B4
:1025B000440E826F94EC0EF004012C0E826F94ECAA
:1025C0000EF01AC0E8FF070BE8CF82F40401300ECA
:1025D000822794EC0EF004012C0E826F94EC0EF026
:1025E000078062EC30F02BC0E8FF003B0043004363
:1025F000030B05EC30F033C182F40401300E822766
:1026000094EC0EF004012C0E826F94EC0EF062EC50
:1026100030F02BC001F1019F019D2CC000F10101A0
:1026200005EC30F02FC182F40401300E822794ECC7
:102630000EF030C182F40401300E822794EC0EF0CB
:1026400031C182F40401300E822794EC0EF032C1C5
:1026500082F40401300E822794EC0EF033C182F430
:102660000401300E822794EC0EF004012C0E826FD0
:1026700094EC0EF062EC30F02DC001F12EC000F1B0
:10268000D89001330033D89001330033010105ECB9
:1026900030F02FC182F40401300E822794EC0EF04A
:1026A00030C182F40401300E822794EC0EF031C167
:1026B00082F40401300E822794EC0EF032C182F4D1
:1026C0000401300E822794EC0EF033C182F4040131
:1026D000300E822794EC0EF08BEF29F0FC0E64ECA8
:1026E0000BF0E8CF0BF003018351520AD8B4A5EFE9
:1026F00013F003018351720AD8B4A8EF13F0030159
:102700008351500AD8B4ABEF13F003018351700A20
:10271000D8B4AEEF13F003018351550AD8B4B1EF2A
:1027200013F003018351750AD8B4B4EF13F0030119
:102730008351430AD8B4BDEF13F003018351630AF8
:10274000D8B4C0EF13F0C9EF13F00B90C3EF13F040
:102750000B80C3EF13F00B92C3EF13F00B82C3EFA8
:1027600013F00B94C3EF13F00B84C3EF13F00B962D
:10277000C3EF13F00B86C3EF13F00B98C3EF13F006
:102780000B88C3EF13F0FC0E0C6E0BC00BF04DEC7E
:102790000BF00401590E826F94EC0EF0119011921F
:1027A00011941198FC0E64EC0BF0E8CF0BF00BA029
:1027B00011800BA211820BA411840BA8118811A007
:1027C000E9EF13F00401520E826F94EC0EF0EEEF7D
:1027D00013F00401720E826F94EC0EF011A8F8EF62
:1027E00013F00401430E826F94EC0EF0FDEF13F032
:1027F0000401630E826F94EC0EF011A207EF14F047
:102800000401500E826F94EC0EF00CEF14F00401F2
:10281000700E826F94EC0EF011A416EF14F0040108
:10282000550E826F94EC0EF01BEF14F00401750E40
:10283000826F94EC0EF08BEF29F004016D0E826F25
:1028400094EC0EF003018351300AD8B475EF14F004
:1028500003018351310AD8B488EF14F00301835186
:10286000320AD8B49BEF14F08DEF29F004014D0E1D
:10287000826F94EC0EF0A3EC30F084C331F185C389
:1028800032F186C333F10101296BB0EC30F027EC53
:1028900030F003018351300AD8B45DEF14F0030126
:1028A0008351310AD8B465EF14F003018351320A21
:1028B000D8B46DEF14F08DEF29F0FD0E0C6E00C151
:1028C0000BF04DEC0BF075EF14F0FE0E0C6E00C12A
:1028D0000BF04DEC0BF088EF14F0FF0E0C6E00C106
:1028E0000BF04DEC0BF09BEF14F00401300E826FF7
:1028F00094EC0EF004012C0E826F94EC0EF062EC5E
:1029000030F0FD0E64EC0BF0E8CF00F1ACEF14F00A
:102910000401310E826F94EC0EF004012C0E826FD4
:1029200094EC0EF062EC30F0FE0E64EC0BF0E8CFAD
:1029300000F1ACEF14F00401320E826F94EC0EF053
:1029400062EC30F004012C0E826F94EC0EF0FF0E5E
:1029500064EC0BF0E8CF00F105EC30F031C182F40B
:102960000401300E822794EC0EF032C182F404018F
:10297000300E822794EC0EF033C182F40401300E45
:10298000822794EC0EF08BEF29F003018351300A7B
:10299000D8B419EF1AF003018351310AD8B446EFC5
:1029A0001BF003018351320AD8B4B4EF1BF00301CA
:1029B0008351330AD8B4C4EF1BF003018351340AA6
:1029C000D8B41FEF1CF003018351350AD8B4E5EFEA
:1029D0001DF003018351360AD8B413EF1EF0030132
:1029E0008351370AD8B4F1EF17F003018351380A45
:1029F000D8B48FEF18F003018351440AD8B41DEF07
:102A000016F003018351640AD8B43DEF16F00301B8
:102A10008351460AD8B4F8EF1CF0030183514D0AE4
:102A2000D8B46AEF16F0030183516D0AD8B484EF6D
:102A300016F0030183515A0AD8B4C0EF1AF003010B
:102A40008351490AD8B413EF1FF003018351500A90
:102A5000D8B445EF1EF003018351540AD8B4BEEF39
:102A60001EF003018351630AD8B4A4EF16F00301EA
:102A70008351430AD8B49CEF17F003018351730AC2
:102A8000D8B4A2EF16F003018351610AD8B46AEFFB
:102A900015F003018351650AD8B469EF1AF00301F8
:102AA0008351450AD8B477EF1AF003018351620AC3
:102AB000D8B485EF1AF003018351420AD8B493EFDA
:102AC0001AF003018351760AD8B4A1EF1AF0D8A402
:102AD0008DEF29F004014C0E826F94EC0EF004018E
:102AE000610E826F94EC0EF0ABEC31F004012C0E11
:102AF000826F94EC0EF062EC30F0AFC500F1010192
:102B000005EC30F031C182F40401300E822794ECE0
:102B10000EF032C182F40401300E822794EC0EF0E4
:102B200033C182F40401300E822794EC0EF00401CC
:102B30002C0E826F94EC0EF062EC30F0B0C500F118
:102B4000010105EC30F031C182F40401300E82271E
:102B500094EC0EF032C182F40401300E822794EC22
:102B60000EF033C182F40401300E822794EC0EF093
:102B700004012C0E826F94EC0EF062EC30F0B1C5C3
:102B800000F1010105EC30F031C182F40401300E96
:102B9000822794EC0EF032C182F40401300E8227B9
:102BA00094EC0EF033C182F40401300E822794ECD1
:102BB0000EF004012C0E826F94EC0EF062EC30F0FB
:102BC000B2C500F1010105EC30F031C182F404011D
:102BD000300E822794EC0EF032C182F40401300EE4
:102BE000822794EC0EF033C182F40401300E822768
:102BF00094EC0EF004012C0E826F94EC0EF062EC5B
:102C000030F0B6C500F1010105EC30F031C182F4BD
:102C10000401300E822794EC0EF032C182F40401DC
:102C2000300E822794EC0EF033C182F40401300E92
:102C3000822794EC0EF041EF1EF003018451300A1C
:102C4000D8B429EF16F003018451310AD8B42DEF1E
:102C500016F0159215962EEF16F01582C70E64EC3D
:102C60000BF0E8CF00F10101008115A20091C70E21
:102C70000C6E00C10BF04DEC0BF0C70E64EC0BF0CA
:102C8000E8CF00F1010100B149EF16F015924AEFCB
:102C900016F0158204014C0E826F94EC0EF00401C4
:102CA000640E826F94EC0EF004012C0E826F94EC93
:102CB0000EF015B263EF16F00401300E826F94EC43
:102CC0000EF068EF16F00401310E826F94EC0EF0F6
:102CD0008BEF29F0A3EC30F084C333F1B0EC30F08B
:102CE00027EC30F0200E0C6E00C10BF04DEC0BF019
:102CF00000C12FF505012F51000A06E005012F51F3
:102D0000010A02E045EC32F004014C0E826F94ECB3
:102D10000EF004014D0E826F94EC0EF004012C0EA7
:102D2000826F94EC0EF062EC30F02FC500F105ECF0
:102D300030F033C182F40401300E822794EC0EF09F
:102D400041EF1EF0FCEF37F004014C0E826F94EC63
:102D50000EF00401630E826F94EC0EF003EC31F080
:102D600004012C0E826F94EC0EF0B9EC16F041EFDA
:102D70001EF062EC30F0B5C500F10101003B0F0E12
:102D8000001705EC30F033C182F40401300E8227C5
:102D900094EC0EF0B5C500F101010F0E0101001712
:102DA00005EC30F033C182F40401300E822794EC3C
:102DB0000EF004012D0E826F94EC0EF0B4C500F1FC
:102DC0000101003B0F0E001705EC30F033C182F417
:102DD0000401300E822794EC0EF0B4C500F101011D
:102DE0000F0E0101001705EC30F033C182F404012D
:102DF000300E822794EC0EF004012D0E826F94ECBD
:102E00000EF0B3C500F10101003B0F0E001705ECF9
:102E100030F033C182F40401300E822794EC0EF0BE
:102E2000B3C500F101010F0E0101001705EC30F0F0
:102E300033C182F40401300E822794EC0EF00401B9
:102E4000200E826F94EC0EF0B2C500F10F0E01015E
:102E5000001705EC30F033C182F40401300E8227F4
:102E600094EC0EF00401200E826F94EC0EF0B1C5CC
:102E700000F101010101003B0F0E001705EC30F0DD
:102E800033C182F40401300E822794EC0EF0B1C5F8
:102E900000F101010F0E0101001705EC30F033C104
:102EA00082F40401300E822794EC0EF004013A0EF5
:102EB000826F94EC0EF0B0C500F10101003B0F0EE3
:102EC000001705EC30F033C182F40401300E822784
:102ED00094EC0EF0B0C500F101010F0E01010017D6
:102EE00005EC30F033C182F40401300E822794ECFB
:102EF0000EF004013A0E826F94EC0EF0AFC500F1B3
:102F00000101003B0F0E001705EC30F033C182F4D5
:102F10000401300E822794EC0EF0AFC500F10101E0
:102F20000F0E001705EC30F033C182F40401300EAF
:102F3000822794EC0EF0120084C3E8FF0F0BE83AEE
:102F4000E8CFB5F585C3E8FF0F0B0501B51387C3BF
:102F5000E8FF0F0BE83AE8CFB4F588C3E8FF0F0BA2
:102F60000501B4138AC3E8FF0F0BE83AE8CFB3F5C5
:102F70008BC3E8FF0F0B0501B3138DC3E8FF0F0BE5
:102F8000E8CFB2F58FC3E8FF0F0BE83AE8CFB1F511
:102F900090C3E8FF0F0B0501B11392C3E8FF0F0BBD
:102FA000E83AE8CFB0F593C3E8FF0F0B0501B01383
:102FB00095C3E8FF0F0BE83AE8CFAFF596C3E8FFFB
:102FC0000F0B0501AF135EEC31F004014C0E826F64
:102FD00094EC0EF00401430E826F94EC0EF0AEEF11
:102FE00016F0078404014C0E826F94EC0EF004017D
:102FF000370E826F94EC0EF004012C0E826F94EC6D
:103000000EF005012E51130A06E005012E51170A94
:103010000DE08CEF18F00101000E006F000E016F43
:10302000100E026F000E036F1FEF18F00101000E6B
:10303000006F000E016F000E026F010E036F05ECB2
:1030400030F02AC182F40401300E822794EC0EF095
:103050002BC182F40401300E822794EC0EF02CC1B7
:1030600082F40401300E822794EC0EF02DC182F41C
:103070000401300E822794EC0EF02EC182F404017C
:10308000300E822794EC0EF02FC182F40401300E32
:10309000822794EC0EF030C182F40401300E8227B6
:1030A00094EC0EF031C182F40401300E822794ECCE
:1030B0000EF032C182F40401300E822794EC0EF03F
:1030C00033C182F40401300E822794EC0EF0040127
:1030D0002C0E826F94EC0EF00101100E006F000EAA
:1030E000016F000E026F000E036F05EC30F031C16E
:1030F00082F40401300E822794EC0EF032C182F487
:103100000401300E822794EC0EF033C182F40401E6
:10311000300E822794EC0EF0079441EF1EF005016B
:10312000216B226B236B246B04014C0E826F94EC99
:103130000EF00401380E826F94EC0EF004012C0E98
:10314000826F94EC0EF00101100E006F000E016F03
:10315000000E026F000E036F05EC30F02AC182F4FE
:103160000401300E822794EC0EF02BC182F404018E
:10317000300E822794EC0EF02CC182F40401300E44
:10318000822794EC0EF02DC182F40401300E8227C8
:1031900094EC0EF02EC182F40401300E822794ECE0
:1031A0000EF02FC182F40401300E822794EC0EF051
:1031B00030C182F40401300E822794EC0EF031C14C
:1031C00082F40401300E822794EC0EF032C182F4B6
:1031D0000401300E822794EC0EF033C182F4040116
:1031E000300E822794EC0EF004012C0E826F94ECCA
:1031F0000EF025C500F126C501F127C502F128C54D
:1032000003F10101100E046F000E056F000E066F32
:10321000000E076F98EC2FF000C133F501C134F5B3
:1032200002C135F503C136F505EC30F02AC182F450
:103230000401300E822794EC0EF02BC182F40401BD
:10324000300E822794EC0EF02CC182F40401300E73
:10325000822794EC0EF02DC182F40401300E8227F7
:1032600094EC0EF02EC182F40401300E822794EC0F
:103270000EF02FC182F40401300E822794EC0EF080
:1032800030C182F40401300E822794EC0EF031C17B
:1032900082F40401300E822794EC0EF032C182F4E5
:1032A0000401300E822794EC0EF033C182F4040145
:1032B000300E822794EC0EF09EEC0EF00501336781
:1032C00069EF19F0346769EF19F0356769EF19F0A4
:1032D000366702D008EF1AF0129E129C21C500F149
:1032E00022C501F123C502F124C503F1899A400EDC
:1032F000C76E200EC66E9E96C69E0B0EC96EFF0E42
:103300009EB602D0E82EFCD79E96C69E02C1C9FF8B
:10331000FF0E9EB602D0E82EFCD79E96C69E01C137
:10332000C9FFFF0E9EB602D0E82EFCD79E96C69E21
:1033300000C1C9FFFF0E9EB602D0E82EFCD79E96B4
:10334000C69EC952FF0E9EB602D0E82EFCD70501DC
:10335000100E326F040114EE00F080517F0BE12655
:103360009E96C69EC952FF0E9EB602D0E82EFCD78E
:10337000C9CFE7FF0401802B0501322FAAEF19F016
:10338000898A33C500F134C501F135C502F136C56E
:1033900003F10101010E046F000E056F000E066FB0
:1033A000000E076F67EC2FF000C133F501C134F553
:1033B00002C135F503C136F505013367E7EF19F0B2
:1033C0003467E7EF19F03567E7EF19F0366702D099
:1033D00008EF1AF021C500F122C501F123C502F161
:1033E00024C503F10101100E046F000E056F000EDD
:1033F000066F000E076F6CEC2FF000C121F501C1C4
:1034000022F502C123F503C124F5128E8DEF29F0B8
:103410000401450E826F94EC0EF004014F0E826F92
:1034200094EC0EF00401460E826F94EC0EF041EF26
:103430001EF007845AEC37F062EC30F02DC500F135
:1034400005EC30F004014C0E826F94EC0EF0040198
:10345000300E826F94EC0EF004012C0E826F94EC0F
:103460000EF031C182F40401300E822794EC0EF08C
:1034700032C182F40401300E822794EC0EF033C185
:1034800082F40401300E822794EC0EF004012C0E1D
:10349000826F94EC0EF062EC30F02EC500F105EC7A
:1034A00030F031C182F40401300E822794EC0EF02A
:1034B00032C182F40401300E822794EC0EF033C145
:1034C00082F40401300E822794EC0EF0079441EF51
:1034D0001EF004014C0E826F94EC0EF00401650E98
:1034E000826F94EC0EF021EC33F041EF1EF00401FA
:1034F0004C0E826F94EC0EF00401450E826F94EC3A
:103500000EF038EC33F041EF1EF004014C0E826FE8
:1035100094EC0EF00401620E826F94EC0EF066ECF7
:1035200033F041EF1EF004014C0E826F94EC0EF06C
:103530000401420E826F94EC0EF04FEC33F041EF39
:103540001EF004014C0E826F94EC0EF00401760E16
:10355000826F94EC0EF004012C0E826F94EC0EF04E
:1035600010A807D00401310E826F94EC0EF041EFE9
:103570001EF00401300E826F94EC0EF041EF1EF04D
:1035800004014C0E826F94EC0EF004015A0E826F0F
:1035900094EC0EF004012C0E826F94EC0EF05AECB9
:1035A00037F062EC30F005012E51130A06E00501F8
:1035B0002E51170A0DE0F1EF1AF00101000E006F15
:1035C000000E016F100E026F000E036FF1EF1AF084
:1035D0000101000E006F000E016F000E026F010E60
:1035E000036F0101100E046F000E056F000E066FD1
:1035F000000E076F98EC2FF005EC30F02AC182F432
:103600000401300E822794EC0EF02BC182F40401E9
:10361000300E822794EC0EF02CC182F40401300E9F
:10362000822794EC0EF02DC182F40401300E822723
:1036300094EC0EF02EC182F40401300E822794EC3B
:103640000EF02FC182F40401300E822794EC0EF0AC
:1036500030C182F40401300E822794EC0EF031C1A7
:1036600082F40401300E822794EC0EF032C182F411
:103670000401300E822794EC0EF033C182F4040171
:10368000300E822794EC0EF041EF1EF00784040107
:103690004C0E826F94EC0EF00401310E826F94ECAC
:1036A0000EF004012C0E826F94EC0EF025C500F193
:1036B00026C501F127C502F128C503F10101100E4D
:1036C000046F000E056F000E066F000E076F98EC7A
:1036D0002FF005EC30F02AC182F40401300E82276D
:1036E00094EC0EF02BC182F40401300E822794EC8E
:1036F0000EF02CC182F40401300E822794EC0EF0FF
:103700002DC182F40401300E822794EC0EF02EC1FC
:1037100082F40401300E822794EC0EF02FC182F463
:103720000401300E822794EC0EF030C182F40401C3
:10373000300E822794EC0EF031C182F40401300E79
:10374000822794EC0EF032C182F40401300E8227FD
:1037500094EC0EF033C182F40401300E822794EC15
:103760000EF0079441EF1EF0078404014C0E826FA7
:1037700094EC0EF00401320E826F94EC0EF055ECD6
:1037800035F0079441EF1EF0078437B0CAEF1BF005
:10379000DDEF1BF0010E166E04014C0E826F94ECEF
:1037A0000EF00401330E826F94EC0EF0B2EC35F0A3
:1037B000000E166E079451EF1BF0020E166EB2EC5F
:1037C00035F08B800501010E306F3C0E316F010129
:1037D0005E6B5F6B606B616B626B636B646B656B85
:1037E000666B676B686B696B536B546BCF6ACE6AA1
:1037F0000F9A0F9C0F9E030E166E04014C0E826FE3
:1038000094EC0EF00401330E826F94EC0EF0040180
:103810002C0E826F94EC0EF004012D0E826F94EC4E
:103820000EF00401310E826F94EC0EF08BEF29F054
:10383000B2EC35F0000E166E8B908DEF29F00784F8
:1038400004014C0E826F94EC0EF00401340E826F72
:1038500094EC0EF004012C0E826F94EC0EF0A3ECAD
:1038600030F084C32AF185C32BF186C32CF187C3C2
:103870002DF188C32EF189C32FF18AC330F18BC398
:1038800031F18CC332F18DC333F10101296BB0ECFE
:1038900030F027EC30F0100E046F000E056F000EB4
:1038A000066F000E076F78EC2FF000C121F501C103
:1038B00022F502C123F503C124F50DEC37F038C51C
:1038C000AFF539C5B0F53AC5B1F53BC5B2F53CC564
:1038D000B3F53DC5B4F53EC5B5F5B9EC16F0040138
:1038E0002C0E826F94EC0EF03FC500F140C501F143
:1038F00041C502F142C503F10101000E046F000E43
:10390000056F010E066F000E076F98EC2FF005ECA7
:1039100030F029678EEF1CF093EF1CF004012D0EA0
:10392000826F94EC0EF030C182F40401300E8227D5
:1039300094EC0EF031C182F40401300E822794EC35
:103940000EF004012E0E826F94EC0EF032C182F460
:103950000401300E822794EC0EF033C182F404018E
:10396000300E822794EC0EF004012C0E826F94EC42
:103970000EF062EC30F043C500F144C501F1B7EC44
:103980002AF004012C0E826F94EC0EF062EC30F001
:1039900045C500F105EC30F031C182F40401300E70
:1039A000822794EC0EF032C182F40401300E82279B
:1039B00094EC0EF033C182F40401300E822794ECB3
:1039C0000EF004012C0E826F94EC0EF037C5E8FF68
:1039D000E8B806D00401300E826F94EC0EF005D0EA
:1039E0000401310E826F94EC0EF0079441EF1EF04B
:1039F000A3EC30F085C32AF186C32BF187C32CF1E9
:103A000088C32DF189C32EF18AC32FF18BC330F106
:103A10008CC331F18DC332F18EC333F10101296BB7
:103A2000B0EC30F027EC30F00101010E046F000E15
:103A3000056F000E066F000E076F67EC2FF0100E7B
:103A4000046F000E056F000E066F000E076F78EC16
:103A50002FF000C129F501C12AF502C12BF503C1E0
:103A60002CF5DCEC34F004014C0E826F94EC0EF07B
:103A70000401460E826F94EC0EF004012C0E826F4E
:103A800094EC0EF025C500F126C501F127C502F121
:103A900028C503F10101100E046F000E056F000E22
:103AA000066F000E076F98EC2FF005EC30F02AC17E
:103AB00082F40401300E822794EC0EF02BC182F4C4
:103AC0000401300E822794EC0EF02CC182F4040124
:103AD000300E822794EC0EF02DC182F40401300EDA
:103AE000822794EC0EF02EC182F40401300E82275E
:103AF00094EC0EF02FC182F40401300E822794EC76
:103B00000EF030C182F40401300E822794EC0EF0E6
:103B100031C182F40401300E822794EC0EF032C1E0
:103B200082F40401300E822794EC0EF033C182F44B
:103B30000401300E822794EC0EF041EF1EF037B0F6
:103B4000A4EF1DF0020E166EB2EC35F00001165017
:103B5000020AD8B4BBEF1DF015B2B6EF1DF081BA62
:103B6000B6EF1DF0000E166E8DEF29F0050E166EE5
:103B70001584FCEF37F08B8001015E6B5F6B606B2F
:103B8000616B626B636B646B656B666B676B686BB9
:103B9000696B536B546BCF6ACE6A0F9A0F9C0F9E62
:103BA000030E166E8DEF29F0B2EC35F015B2E0EF92
:103BB0001DF081BAE0EF1DF0000E166E8DEF29F0BA
:103BC000050E166E1584FCEF37F004014C0E826F63
:103BD00094EC0EF00401350E826F94EC0EF00401AB
:103BE0002C0E826F94EC0EF062EC30F00784B9C5B5
:103BF00000F1079405EC30F031C182F40401300E7D
:103C0000822794EC0EF032C182F40401300E822738
:103C100094EC0EF033C182F40401300E822794EC50
:103C20000EF041EF1EF075EC35F062EC30F037C568
:103C300000F105EC30F004014C0E826F94EC0EF0B4
:103C40000401360E826F94EC0EF004012C0E826F8C
:103C500094EC0EF031C182F40401300E822794EC12
:103C60000EF032C182F40401300E822794EC0EF083
:103C700033C182F40401300E822794EC0EF041EF40
:103C80001EF09EEC0EF08DEF29F004014C0E826FB9
:103C900094EC0EF00401500E826F94EC0EF00401CF
:103CA0002C0E826F94EC0EF085C32AF186C32BF1A3
:103CB00087C32CF188C32DF189C32EF18AC32FF15C
:103CC0008BC330F18CC331F18DC332F18EC333F12C
:103CD0000101B0EC30F027EC30F003018451530ABD
:103CE0000DE0030184514D0A38E00401780E826F23
:103CF00094EC0EF09EEC0EF08DEF29F00401530EC3
:103D0000826F94EC0EF0250E0C6E00C10BF04DECA2
:103D10000BF0260E0C6E01C10BF04DEC0BF0270ED4
:103D20000C6E02C10BF04DEC0BF0280E0C6E03C1B3
:103D30000BF04DEC0BF000C157F501C158F502C175
:103D400059F503C15AF500C15BF501C15CF502C12B
:103D50005DF503C15EF522EF1FF004014D0E826F89
:103D600094EC0EF0290E0C6E00C10BF04DEC0BF034
:103D700000C15FF500C160F522EF1FF004014C0E99
:103D8000826F94EC0EF00401540E826F94EC0EF0EE
:103D900004012C0E826F94EC0EF084C32AF185C3CB
:103DA0002BF186C32CF187C32DF188C32EF189C373
:103DB0002FF18AC330F18BC331F18DC332F18EC341
:103DC00033F10101B0EC30F027EC30F00101000ECE
:103DD000046F000E056F010E066F000E076F78EC82
:103DE0002FF0210E0C6E00C10BF04DEC0BF0220EEB
:103DF0000C6E01C10BF04DEC0BF0230E0C6E02C1EA
:103E00000BF04DEC0BF0240E0C6E03C10BF04DECDF
:103E10000BF000C161F501C162F502C163F503C198
:103E200064F522EF1FF004014C0E826F94EC0EF04B
:103E30000401490E826F94EC0EF004012C0E826F87
:103E400094EC0EF0250E64EC0BF0E8CF00F1260E9A
:103E500064EC0BF0E8CF01F1270E64EC0BF0E8CF37
:103E600002F1280E64EC0BF0E8CF03F105EC30F022
:103E7000C8EC2DF00401730E826F94EC0EF0040177
:103E80002C0E826F94EC0EF062EC30F0290E64EC94
:103E90000BF0E8CF00F105EC30F0C8EC2DF0040198
:103EA0006D0E826F94EC0EF004012C0E826F94EC78
:103EB0000EF05BC500F15CC501F15DC502F15EC5A8
:103EC00003F105EC30F0C8EC2DF00401730E826FA5
:103ED00094EC0EF004012C0E826F94EC0EF062EC68
:103EE00030F060C500F105EC30F0C8EC2DF00401B5
:103EF0006D0E826F94EC0EF004012C0E826F94EC28
:103F00000EF061C500F162C501F163C502F164C53F
:103F100003F1A8EC29F004012C0E826F94EC0EF052
:103F20009EEC0EF08DEF29F083C32AF184C32BF1B0
:103F300085C32CF186C32DF187C32EF188C32FF1E1
:103F400089C330F18AC331F18BC332F18CC333F1B1
:103F50000101B0EC30F027EC30F0160E0C6E00C111
:103F60000BF04DEC0BF0170E0C6E01C10BF04DEC8D
:103F70000BF0180E0C6E02C10BF04DEC0BF0190E8D
:103F80000C6E03C10BF04DEC0BF000C18EF101C1C2
:103F90008FF102C190F103C191F100C192F101C111
:103FA00093F102C194F103C195F176EF20F083C340
:103FB0002AF184C32BF185C32CF186C32DF187C36D
:103FC0002EF188C32FF189C330F18AC331F18BC33D
:103FD00032F18CC333F10101B0EC30F027EC30F05A
:103FE00000C18EF101C18FF102C190F103C191F1C5
:103FF00000C192F101C193F102C194F103C195F1A5
:1040000076EF20F083C32AF184C32BF185C32CF112
:1040100086C32DF187C32EF188C32FF189C330F1F8
:104020008AC331F18CC332F18DC333F10101B0EC9D
:1040300030F027EC30F00101000E046F000E056F28
:10404000010E066F000E076F78EC2FF01A0E0C6E43
:1040500000C10BF04DEC0BF01B0E0C6E01C10BF010
:104060004DEC0BF01C0E0C6E02C10BF04DEC0BF086
:104070001D0E0C6E03C10BF04DEC0BF000C196F160
:1040800001C197F102C198F103C199F176EF20F0D7
:1040900083C32AF184C32BF185C32CF186C32DF190
:1040A00087C32EF188C32FF189C330F18AC331F160
:1040B0008CC332F18DC333F10101B0EC30F027EC49
:1040C00030F00101000E046F000E056F010E066F47
:1040D000000E076F78EC2FF000C196F101C197F147
:1040E00002C198F103C199F176EF20F0160E64EC4D
:1040F0000BF0E8CF00F1170E64EC0BF0E8CF01F104
:10410000180E64EC0BF0E8CF02F1190E64EC0BF022
:10411000E8CF03F105EC30F0C8EC2DF00401730E8C
:10412000826F94EC0EF004012C0E826F94EC0EF072
:104130008EC100F18FC101F190C102F191C103F173
:1041400005EC30F0C8EC2DF00401730E826F94EC96
:104150000EF004012C0E826F94EC0EF01A0E64EC3B
:104160000BF0E8CF00F11B0E64EC0BF0E8CF01F18F
:104170001C0E64EC0BF0E8CF02F11D0E64EC0BF0AA
:10418000E8CF03F1A8EC29F004012C0E826F94EC27
:104190000EF096C100F197C101F198C102F199C1E9
:1041A00003F1A8EC29F09EEC0EF08DEF29F004014C
:1041B000690E826F94EC0EF004012C0E826F94EC69
:1041C0000EF00101040E006F000E016F000E026F71
:1041D000000E036F05EC30F02CC182F40401300EA8
:1041E000822794EC0EF02DC182F40401300E822758
:1041F00094EC0EF02EC182F40401300E822794EC70
:104200000EF02FC182F40401300E822794EC0EF0E0
:1042100030C182F40401300E822794EC0EF031C1DB
:1042200082F40401300E822794EC0EF032C182F445
:104230000401300E822794EC0EF033C182F40401A5
:10424000300E822794EC0EF004012C0E826F94EC59
:104250000EF00101060E006F000E016F000E026FDE
:10426000000E036F05EC30F02CC182F40401300E17
:10427000822794EC0EF02DC182F40401300E8227C7
:1042800094EC0EF02EC182F40401300E822794ECDF
:104290000EF02FC182F40401300E822794EC0EF050
:1042A00030C182F40401300E822794EC0EF031C14B
:1042B00082F40401300E822794EC0EF032C182F4B5
:1042C0000401300E822794EC0EF033C182F4040115
:1042D000300E822794EC0EF004012C0E826F94ECC9
:1042E0000EF00101450E006F000E016F000E026F0F
:1042F000000E036F05EC30F02CC182F40401300E87
:10430000822794EC0EF02DC182F40401300E822736
:1043100094EC0EF02EC182F40401300E822794EC4E
:104320000EF02FC182F40401300E822794EC0EF0BF
:1043300030C182F40401300E822794EC0EF031C1BA
:1043400082F40401300E822794EC0EF032C182F424
:104350000401300E822794EC0EF033C182F4040184
:10436000300E822794EC0EF004012C0E826F94EC38
:104370000EF0200EF86EF76AF66A04010900F5CF18
:1043800082F494EC0EF00900F5CF82F494EC0EF078
:104390000900F5CF82F494EC0EF00900F5CF82F419
:1043A00094EC0EF00900F5CF82F494EC0EF00900C5
:1043B000F5CF82F494EC0EF00900F5CF82F494EC82
:1043C0000EF00900F5CF82F494EC0EF09EEC0EF0A6
:1043D0008DEF29F08351630AD8A48BEF29F0845123
:1043E000610AD8A48BEF29F085516C0AD8A48BEF11
:1043F00029F08651410A3FE08651440A1BE086516C
:10440000420AD8B44EEF22F08651350AD8B417EFDD
:104410002BF08651360AD8B46CEF2BF08651370A50
:10442000D8B4D5EF2BF08651380AD8B433EF2CF03E
:104430008BEF29F00798079A04017A0E826F94ECAB
:104440000EF00401780E826F94EC0EF00401640EFD
:10445000826F94EC0EF00401550E826F94EC0EF016
:1044600037EF22F004014C0E826F94EC0EF09EECBC
:104470000EF08DEF29F00788079A04017A0E826FFB
:1044800094EC0EF00401410E826F94EC0EF00401E6
:10449000610E826F94EC0EF02BEF22F00798078AE2
:1044A00004017A0E826F94EC0EF00401420E826FCA
:1044B00094EC0EF00401610E826F94EC0EF02BEF81
:1044C00022F0010166676CEF22F067676CEF22F063
:1044D00068676CEF22F0696716D001014F6778EFCB
:1044E00022F0506778EF22F0516778EF22F05267A0
:1044F0000AD00101000E006F000E016F000E026F66
:10450000000E036F120011B80AD00101620E046F91
:10451000010E056F000E066F000E076F09D0010136
:10452000A70E046F020E056F000E066F000E076FD8
:1045300066C100F167C101F168C102F169C103F10F
:1045400067EC2FF003BF15EF23F0119A119C0101C6
:10455000000E046FA80E056F550E066F020E076F52
:1045600066C100F167C101F168C102F169C103F1DF
:1045700066C18AF167C18BF168C18CF169C18DF1A7
:1045800067EC2FF003BF0BD00101000E8A6FA80E5D
:104590008B6F550E8C6F020E8D6F118A119C0E0E53
:1045A00064EC0BF0E8CF18F10F0E64EC0BF0E8CFE1
:1045B00019F1100E64EC0BF0E8CF1AF1110E64EC57
:1045C0000BF0E8CF1BF1B0EC2EF08AC104F18BC1E7
:1045D00005F18CC106F18DC107F167EC2FF0078260
:1045E00074EC2EF0B0EC2EF0079274EC2EF08AC131
:1045F00000F18BC101F18CC102F18DC103F1079271
:1046000074EC2EF0CC0E046FE00E056F870E066F73
:10461000050E076F67EC2FF000C118F101C119F109
:1046200002C11AF103C11BF140D013AA1AEF23F003
:10463000138E139A119C119A0101800E006F1A0EAD
:10464000016F060E026F000E036F4FC104F150C1DF
:1046500005F151C106F152C107F167EC2FF003AF2C
:1046600005D062EC30F0118C119A12000E0E64EC41
:104670000BF0E8CF18F10F0E64EC0BF0E8CF19F156
:10468000100E64EC0BF0E8CF1AF1110E64EC0BF095
:10469000E8CF1BF14FC100F150C101F151C102F14E
:1046A00052C103F1078274EC2EF018C100F119C158
:1046B00001F11AC102F11BC103F112000784BAC152
:1046C00066F1BBC167F1BCC168F1BDC169F14BC105
:1046D0004FF14CC150F14DC151F14EC152F157C192
:1046E00059F158C15AF10794010166677FEF23F031
:1046F00067677FEF23F068677FEF23F0696716D065
:1047000001014F678BEF23F050678BEF23F0516768
:104710008BEF23F052670AD00101000E006F000EEC
:10472000016F000E026F000E036F120011B80AD065
:104730000101620E046F010E056F000E066F000E80
:10474000076F09D00101A70E046F020E056F000E5E
:10475000066F000E076F66C100F167C101F168C105
:1047600002F169C103F167EC2FF003BF17EF24F0EA
:104770000101000E046FA80E056F550E066F020EA4
:10478000076F66C100F167C101F168C102F169C13B
:1047900003F166C18AF167C18BF168C18CF169C10F
:1047A0008DF167EC2FF003BF09D00101000E8A6F75
:1047B000A80E8B6F550E8C6F020E8D6FB0EC2EF025
:1047C00000C104F101C105F102C106F103C107F105
:1047D000000E006FA00E016F980E026F7B0E036F2C
:1047E00098EC2FF000C118F101C119F102C11AF1C2
:1047F00003C11BF1000E006FA00E016F980E026F37
:104800007B0E036F8AC104F18BC105F18CC106F1E7
:104810008DC107F198EC2FF018C104F119C105F111
:104820001AC106F11BC107F167EC2FF0120001015C
:10483000A80E006F610E016F000E026F000E036F75
:104840004FC104F150C105F151C106F152C107F148
:1048500067EC2FF003AF0AD00101A80E006F610EC4
:10486000016F000E026F000E036F00D0C80E006FC4
:10487000AF0E016F000E026F000E036F4FC104F107
:1048800050C105F151C106F152C107F178EC2FF08A
:1048900012000401730E826F94EC0EF004012C0ED2
:1048A000826F94EC0EF0078462C166F163C167F118
:1048B00064C168F165C169F14BC14FF14CC150F160
:1048C0004DC151F14EC152F157C159F158C15AF180
:1048D00007946FEC24F09EEC0EF08DEF29F066C18A
:1048E00000F167C101F168C102F169C103F1010181
:1048F00005EC30F0C8EC2DF00401630E826F94ECEF
:104900000EF004012C0E826F94EC0EF04FC100F1FA
:1049100050C101F151C102F152C103F1010105EC95
:1049200030F0C8EC2DF00401660E826F94EC0EF0AE
:1049300004012C0E826F94EC0EF062EC30F059C141
:1049400000F15AC101F1010105EC30F0C8EC2DF085
:104950000401740E826F94EC0EF0120010820401B8
:10496000530E826F94EC0EF004012C0E826F94ECC7
:104970000EF083C32AF184C32BF185C32CF186C3C7
:104980002DF187C32EF188C32FF189C330F18AC37B
:1049900031F18BC332F18CC333F10101B0EC30F053
:1049A00027EC30F000C166F101C167F102C168F186
:1049B00003C169F18EC32AF18FC32BF190C32CF18F
:1049C00091C32DF192C32EF193C32FF194C330F113
:1049D00095C331F196C332F197C333F10101B0ECC5
:1049E00030F027EC30F000C14FF101C150F102C1AD
:1049F00051F103C152F1A3EC30F099C32FF19AC3E6
:104A000030F19BC331F19CC332F19DC333F10101FD
:104A1000B0EC30F027EC30F000C159F101C15AF18F
:104A20006FEC24F004012C0E826F94EC0EF029EF51
:104A300025F0118E1CA002D01CAE108C1BBE02D023
:104A40001BA4108E03018251520A02E10F8201D091
:104A50000F928251750A02E1108401D010948251A4
:104A6000550A02E1108601D010968351310A03E104
:104A70001382138402D01392139403018351660AA4
:104A800001E056D00401660E826F94EC0EF0040132
:104A90002C0E826F94EC0EF05EEC23F005EC30F0FF
:104AA0002AC182F40401300E822794EC0EF02BC14F
:104AB00082F40401300E822794EC0EF02CC182F4B3
:104AC0000401300E822794EC0EF02DC182F4040113
:104AD000300E822794EC0EF02EC182F40401300EC9
:104AE000822794EC0EF02FC182F40401300E82274D
:104AF00094EC0EF030C182F40401300E822794EC65
:104B00000EF031C182F40401300E822794EC0EF0D5
:104B100032C182F40401300E822794EC0EF033C1CE
:104B200082F40401300E822794EC0EF08BEF29F012
:104B300011A003D011A401D01084078410B202EF99
:104B400026F010A4E6EF25F0BAC166F1BBC167F10B
:104B5000BCC168F1BDC169F1BEC16AF1BFC16BF1F1
:104B6000C0C16CF1C1C16DF1C2C16EF1C3C16FF1C1
:104B7000C4C170F1C5C171F1C6C172F1C7C173F191
:104B8000C8C174F1C9C175F1CAC176F1CBC177F161
:104B9000CCC178F1CDC179F1CEC17AF1CFC17BF131
:104BA000D0C17CF1D1C17DF1D2C17EF1D3C17FF101
:104BB000D4C180F1D5C181F1D6C182F1D7C183F1D1
:104BC000D8C184F1D9C185F1EEEF25F062C166F15B
:104BD00063C167F164C168F165C169F1BAC186F169
:104BE000BBC187F1BCC188F1BDC189F14BC14FF197
:104BF0004CC150F14DC151F14EC152F157C159F163
:104C000058C15AF107940FA024EF26F001019667CE
:104C100011EF26F0976711EF26F0986711EF26F055
:104C2000996715EF26F024EF26F061EC22F096C18B
:104C300004F197C105F198C106F199C107F167EC3C
:104C40002FF003BF51EF29F061EC22F00101000EBB
:104C5000046F000E056F010E066F000E076F98ECD3
:104C60002FF011A02AD011A228D005EC30F029672E
:104C700001D005D004012D0E826F94EC0EF030C1EE
:104C800082F40401300E822794EC0EF031C182F4DC
:104C90000401300E822794EC0EF032C182F404013C
:104CA000300E822794EC0EF033C182F40401300EF2
:104CB000822794EC0EF09EEC0EF012A8C5D012984C
:104CC0001DC01EF01E3A1E42070E1E1600011E5089
:104CD000000AD8B4F0EF26F000011E50010AD8B443
:104CE0007CEF26F000011E50020AD8B47AEF26F0BD
:104CF00022EF27F022EF27F062EC30F02DC001F117
:104D00002EC000F1D89001330033D8900133003326
:104D10000101630E046F000E056F000E066F000E9A
:104D2000076F98EC2FF0280E046F000E056F000E31
:104D3000066F000E076F67EC2FF000C130F062ECD9
:104D400030F02BC001F1019F019D2CC000F1010149
:104D5000A40E046F000E056F000E066F000E076FA5
:104D600098EC2FF000C12FF000C104F101C105F152
:104D700002C106F103C107F1640E006F000E016F5E
:104D8000000E026F000E036F67EC2FF0050E046F2C
:104D9000000E056F000E066F000E076F98EC2FF0E7
:104DA00000C104F101C105F102C106F103C107F11F
:104DB00062EC30F030C000F167EC2FF000C131F050
:104DC00031C0E8FF050F305C03E78A8422EF27F04B
:104DD00031C0E8FF0A0F305C01E68A9422EF27F029
:104DE00000C124F101C125F102C126F103C127F15F
:104DF00062EC30F068EC30F01D501F0BE8CF00F192
:104E00000101640E046F000E056F000E066F000EA8
:104E1000076F78EC2FF024C104F125C105F126C1FC
:104E200006F127C107F167EC2FF003BF02D08A9487
:104E300001D08A8424C100F125C101F126C102F10B
:104E400027C103F18DEF29F000C124F101C125F143
:104E500002C126F103C127F110AE4DD0109E00C152
:104E600008F101C109F102C10AF103C10BF105EC1E
:104E700030F030C1E2F131C1E3F132C1E4F133C1CC
:104E8000E5F108C100F109C101F10AC102F10BC14C
:104E900003F101016C0E046F070E056F000E066F23
:104EA000000E076F67EC2FF003BF04D00101550E11
:104EB000E66F1CD008C100F109C101F10AC102F17D
:104EC0000BC103F10101A40E046F060E056F000E65
:104ED000066F000E076F67EC2FF003BF04D00101CF
:104EE0007F0EE66F03D00101FF0EE66F1F8E11AE3D
:104EF00051EF29F0119E24C100F125C101F126C115
:104F000002F127C103F111A005D011A203D00FB007
:104F100051EF29F010A494EF27F00401750E826F71
:104F200094EC0EF099EF27F00401720E826F94EC6E
:104F30000EF004012C0E826F94EC0EF005EC30F0B4
:104F40002967A8EF27F00401200E826FABEF27F04E
:104F500004012D0E826F94EC0EF030C182F4040136
:104F6000300E822794EC0EF031C182F40401300E31
:104F7000822794EC0EF004012E0E826F94EC0EF05A
:104F800032C182F40401300E822794EC0EF033C15A
:104F900082F40401300E822794EC0EF004016D0EB1
:104FA000826F94EC0EF004012C0E826F94EC0EF0E4
:104FB0004FC100F150C101F151C102F152C103F1E1
:104FC000010105EC30F0C8EC2DF00401480E826FB1
:104FD00094EC0EF004017A0E826F94EC0EF0040152
:104FE0002C0E826F94EC0EF066C100F167C101F1E6
:104FF00068C102F169C103F1010105EC30F0C8ECB0
:105000002DF00401630E826F94EC0EF004012C0E5F
:10501000826F94EC0EF066C100F167C101F168C1C6
:1050200002F169C103F101010A0E046F000E056F60
:10503000000E066F000E076F78EC2FF0000E046F65
:10504000120E056F000E066F000E076F98EC2FF022
:1050500005EC30F02AC182F40401300E822794EC72
:105060000EF02BC182F40401300E822794EC0EF076
:105070002CC182F40401300E822794EC0EF02DC175
:1050800082F40401300E822794EC0EF02EC182F4DB
:105090000401300E822794EC0EF02FC182F404013B
:1050A000300E822794EC0EF030C182F40401300EF1
:1050B000822794EC0EF004012E0E826F94EC0EF019
:1050C00031C182F40401300E822794EC0EF032C11B
:1050D00082F40401300E822794EC0EF033C182F486
:1050E0000401300E822794EC0EF00401730E826FDF
:1050F00094EC0EF004012C0E826F94EC0EF062EC36
:1051000030F059C100F15AC101F1B7EC2AF013A2F5
:10511000D9EF28F004012C0E826F94EC0EF086C1BA
:1051200066F187C167F188C168F189C169F161ECF5
:1051300022F00101000E046F000E056F010E066FD4
:10514000000E076F98EC2FF005EC30F02967AEEFFA
:1051500028F00401200E826FB1EF28F004012D0E1B
:10516000826F94EC0EF030C182F40401300E82277D
:1051700094EC0EF031C182F40401300E822794ECDD
:105180000EF004012E0E826F94EC0EF032C182F408
:105190000401300E822794EC0EF033C182F4040136
:1051A000300E822794EC0EF004016D0E826F94ECA9
:1051B0000EF013A400EF29F004012C0E826F94EC82
:1051C0000EF013ACEEEF28F00401500E826F94EC59
:1051D0000EF0139C1398139A00EF29F013AEFBEF17
:1051E00028F00401460E826F94EC0EF0139E139883
:1051F000139A00EF29F00401530E826F94EC0EF025
:1052000037B017EF29F004012C0E826F94EC0EF0EA
:105210008BB012EF29F00401440E826F94EC0EF073
:1052200017EF29F00401530E826F94EC0EF00FB2C9
:105230001DEF29F00FA04FEF29F004012C0E826F13
:1052400094EC0EF0200EF86EF76AF66A040109007D
:10525000F5CF82F494EC0EF00900F5CF82F494ECD3
:105260000EF00900F5CF82F494EC0EF00900F5CFB2
:1052700082F494EC0EF00900F5CF82F494EC0EF079
:105280000900F5CF82F494EC0EF00900F5CF82F41A
:1052900094EC0EF00900F5CF82F494EC0EF09EEC45
:1052A0000EF00F90109E12988DEF29F00401630EFE
:1052B000826F94EC0EF004012C0E826F94EC0EF0D1
:1052C00093EC29F004012C0E826F94EC0EF006ECA6
:1052D0002AF004012C0E826F94EC0EF082EC2AF07E
:1052E00004012C0E826F94EC0EF00101F80E006F99
:1052F000CD0E016F660E026F030E036FA8EC29F04E
:1053000004012C0E826F94EC0EF098EC2AF09EECC7
:105310000EF08DEF29F09EEC0EF00301C26B0790AA
:1053200010929CEF2CF0D8900E0E64EC0BF0E8CFAE
:1053300000F10F0E64EC0BF0E8CF01F1100E64ECFD
:105340000BF0E8CF02F1110E64EC0BF0E8CF03F1A3
:105350000101000E046F000E056F010E066F000EB6
:10536000076F98EC2FF005EC30F02AC182F40401AD
:10537000300E822794EC0EF02BC182F40401300E23
:10538000822794EC0EF02CC182F40401300E8227A7
:1053900094EC0EF02DC182F40401300E822794ECBF
:1053A0000EF02EC182F40401300E822794EC0EF030
:1053B0002FC182F40401300E822794EC0EF030C12C
:1053C00082F40401300E822794EC0EF031C182F495
:1053D0000401300E822794EC0EF004012E0E826F31
:1053E00094EC0EF032C182F40401300E822794EC6A
:1053F0000EF033C182F40401300E822794EC0EF0DB
:1054000004016D0E826F94EC0EF01200120E64EC2B
:105410000BF0E8CF00F1130E64EC0BF0E8CF01F1D4
:10542000140E64EC0BF0E8CF02F1150E64EC0BF0F7
:10543000E8CF03F101010A0E046F000E056F000EA4
:10544000066F000E076F78EC2FF0000E046F120E3F
:10545000056F000E066F000E076F98EC2FF005EC3D
:1054600030F02AC182F40401300E822794EC0EF051
:105470002BC182F40401300E822794EC0EF02CC173
:1054800082F40401300E822794EC0EF02DC182F4D8
:105490000401300E822794EC0EF02EC182F4040138
:1054A000300E822794EC0EF02FC182F40401300EEE
:1054B000822794EC0EF030C182F40401300E822772
:1054C00094EC0EF004012E0E826F94EC0EF031C1BC
:1054D00082F40401300E822794EC0EF032C182F483
:1054E0000401300E822794EC0EF033C182F40401E3
:1054F000300E822794EC0EF00401730E826F94EC50
:105500000EF012000A0E64EC0BF0E8CF00F10B0E67
:1055100064EC0BF0E8CF01F10C0E64EC0BF0E8CF7B
:1055200002F10D0E64EC0BF0E8CF03F1B7EF2AF0B7
:10553000060E64EC0BF0E8CF00F1070E64EC0BF004
:10554000E8CF01F1080E64EC0BF0E8CF02F1090E90
:1055500064EC0BF0E8CF03F1B7EF2AF0010162EC45
:1055600030F0078457C100F158C101F107940101DF
:10557000E80E046F800E056F000E066F000E076FB9
:1055800078EC2FF0000E046F040E056F000E066F0E
:10559000000E076F98EC2FF0880E046F130E056F46
:1055A000000E066F000E076F67EC2FF00A0E046FF7
:1055B000000E056F000E066F000E076F98EC2FF0BF
:1055C00005EC30F001012967EBEF2AF00401200E11
:1055D000826FEEEF2AF004012D0E826F94EC0EF034
:1055E00030C182F40401300E822794EC0EF031C1F8
:1055F00082F40401300E822794EC0EF032C182F462
:105600000401300E822794EC0EF004012E0E826FFE
:1056100094EC0EF033C182F40401300E822794EC36
:105620000EF00401430E826F94EC0EF0120087C35B
:105630002AF188C32BF189C32CF18AC32DF18BC3C6
:105640002EF18CC32FF18DC330F18EC331F190C395
:1056500032F191C333F10101296BB0EC30F027EC4A
:1056600030F00101000E046F000E056F010E066F91
:10567000000E076F78EC2FF00E0E0C6E00C10BF0D1
:105680004DEC0BF00F0E0C6E01C10BF04DEC0BF05E
:10569000100E0C6E02C10BF04DEC0BF0110E0C6EE7
:1056A00003C10BF04DEC0BF004017A0E826F94EC09
:1056B0000EF004012C0E826F94EC0EF00401350EF6
:1056C000826F94EC0EF004012C0E826F94EC0EF0BD
:1056D00093EC29F037EF22F087C32AF188C32BF12E
:1056E00089C32CF18AC32DF18BC32EF18CC32FF10A
:1056F0008DC330F18EC331F190C332F191C333F1D8
:105700000101296BB0EC30F027EC30F0880E046F0B
:10571000130E056F000E066F000E076F6CEC2FF076
:10572000000E046F040E056F000E066F000E076F6B
:1057300078EC2FF00101E80E046F800E056F000E6B
:10574000066F000E076F98EC2FF00A0E0C6E00C16A
:105750000BF04DEC0BF00B0E0C6E01C10BF04DEC91
:105760000BF00C0E0C6E02C10BF04DEC0BF00D0E9D
:105770000C6E03C10BF04DEC0BF004017A0E826F3E
:1057800094EC0EF004012C0E826F94EC0EF00401E8
:10579000360E826F94EC0EF004012C0E826F94ECA6
:1057A0000EF082EC2AF037EF22F087C32AF188C38B
:1057B0002BF189C32CF18AC32DF18BC32EF18CC33D
:1057C0002FF18DC330F18FC331F190C332F191C30A
:1057D00033F10101B0EC30F027EC30F0000E046F33
:1057E000120E056F000E066F000E076F78EC2FF09B
:1057F00001010A0E046F000E056F000E066F000E09
:10580000076F98EC2FF0120E0C6E00C10BF04DECF0
:105810000BF0130E0C6E01C10BF04DEC0BF0140EDF
:105820000C6E02C10BF04DEC0BF0150E0C6E03C1AB
:105830000BF04DEC0BF004017A0E826F94EC0EF03D
:1058400004012C0E826F94EC0EF00401370E826F6F
:1058500094EC0EF004012C0E826F94EC0EF006EC2A
:105860002AF037EF22F087C32AF188C32BF189C3CE
:105870002CF18AC32DF18BC32EF18CC32FF18DC374
:1058800030F18EC331F190C332F191C333F1010194
:10589000296BB0EC30F027EC30F0880E046F130E5B
:1058A000056F000E066F000E076F6CEC2FF0000EF8
:1058B000046F040E056F000E066F000E076F78EC84
:1058C0002FF00101E80E046F800E056F000E066FC9
:1058D000000E076F98EC2FF0060E0C6E00C10BF057
:1058E0004DEC0BF0070E0C6E01C10BF04DEC0BF004
:1058F000080E0C6E02C10BF04DEC0BF0090E0C6E95
:1059000003C10BF04DEC0BF004017A0E826F94ECA6
:105910000EF004012C0E826F94EC0EF00401380E90
:10592000826F94EC0EF004012C0E826F94EC0EF05A
:1059300098EC2AF037EF22F007A80FEF2DF00101C5
:10594000800E006F1A0E016F060E026F000E036FBD
:105950004BC104F14CC105F14DC106F14EC107F137
:1059600067EC2FF003BF55EF2DF0C2EC2DF04BC1CB
:1059700000F14CC101F14DC102F14EC103F10782AA
:1059800074EC2EF018C104F119C105F11AC106F129
:105990001BC107F1F80E006FCD0E016F660E026F8E
:1059A000030E036F67EC2FF00E0E0C6E00C10BF0B0
:1059B0004DEC0BF00F0E0C6E01C10BF04DEC0BF02B
:1059C000100E0C6E02C10BF04DEC0BF0110E0C6EB4
:1059D00003C10BF04DEC0BF00784010162EC30F0D9
:1059E00057C100F158C101F107940A0E0C6E00C1B5
:1059F0000BF04DEC0BF00B0E0C6E01C10BF04DECEF
:105A00000BF00C0E0C6E02C10BF04DEC0BF00D0EFA
:105A10000C6E03C10BF04DEC0BF055EF2DF007AA07
:105A200055EF2DF00784010162EC30F057C100F111
:105A300058C101F10794060E0C6E00C10BF04DEC3D
:105A40000BF0070E0C6E01C10BF04DEC0BF0080EC5
:105A50000C6E02C10BF04DEC0BF0090E0C6E03C185
:105A60000BF04DEC0BF0078462C100F163C101F152
:105A700064C102F165C103F10794120E0C6E00C1FE
:105A80000BF04DEC0BF0130E0C6E01C10BF04DEC56
:105A90000BF0140E0C6E02C10BF04DEC0BF0150E5A
:105AA0000C6E03C10BF04DEC0BF00798079A040144
:105AB000805181197F0B0DE09EA8FED714EE00F0F7
:105AC00081517F0BE126E750812B0F01AD6E57EF1F
:105AD0002DF005012F51010A14E081BA75EF2DF068
:105AE00015B28AEF2DF081EF2DF005012F51000A3C
:105AF000D8B4FCEF37F000011650050AD8B4FCEF1B
:105B000037F081B88AEF2DF0ABEC31F0A9EC32F030
:105B100099EC37F0C2EF0DF018C100F119C101F195
:105B20001AC102F11BC103F1000E046F000E056FD4
:105B3000010E066F000E076F98EC2FF029A1B7EF4A
:105B40002DF02051D8B4B7EF2DF018C100F119C1D4
:105B500001F11AC102F11BC103F1000E046F000E26
:105B6000056F0A0E066F000E076F98EC2FF01200FB
:105B7000010104510013055101130651021307518D
:105B8000031312000101186B196B1A6B1B6B1200C7
:105B90002AC182F40401300E822794EC0EF02BC14E
:105BA00082F40401300E822794EC0EF02CC182F4B2
:105BB0000401300E822794EC0EF02DC182F4040112
:105BC000300E822794EC0EF02EC182F40401300EC8
:105BD000822794EC0EF02FC182F40401300E82274C
:105BE00094EC0EF030C182F40401300E822794EC64
:105BF0000EF031C182F40401300E822794EC0EF0D5
:105C000032C182F40401300E822794EC0EF033C1CD
:105C100082F40401300E822794EC0EF012002FC1A2
:105C200082F40401300E822794EC0EF030C182F42D
:105C30000401300E822794EC0EF031C182F404018D
:105C4000300E822794EC0EF032C182F40401300E43
:105C5000822794EC0EF033C182F40401300E8227C7
:105C600094EC0EF01200060E216E060E226E060E49
:105C7000236E212E39EF2EF0222E39EF2EF0232E17
:105C800039EF2EF08B84020E216E020E226E020E70
:105C9000236E212E49EF2EF0222E49EF2EF0232ED7
:105CA00049EF2EF08B941200FF0E226E22C023F0DB
:105CB000030E216E8B84212E5AEF2EF0030E216EDF
:105CC000232E5AEF2EF08B9422C023F0030E216E68
:105CD000212E68EF2EF0030E216E233E68EF2EF08A
:105CE000222E56EF2EF012000101005305E1015360
:105CF00003E1025301E1002B37EC2FF062EC30F0AE
:105D00003951006F3A51016F420E046F4B0E056F0F
:105D1000000E066F000E076F78EC2FF000C104F143
:105D200001C105F102C106F103C107F118C100F17B
:105D300019C101F11AC102F11BC103F107B2A5EFAC
:105D40002EF06CEC2FF0A7EF2EF067EC2FF000C1D7
:105D500018F101C119F102C11AF103C11BF11200BE
:105D600062EC30F059C100F15AC101F1060E64EC49
:105D70000BF0E8CF04F1070E64EC0BF0E8CF05F16F
:105D8000080E64EC0BF0E8CF06F1090E64EC0BF0A2
:105D9000E8CF07F167EC2FF000C124F101C125F134
:105DA00002C126F103C127F1290E046F000E056F11
:105DB000000E066F000E076F78EC2FF0EE0E046FEA
:105DC000430E056F000E066F000E076F6CEC2FF090
:105DD00024C104F125C105F126C106F127C107F14F
:105DE00078EC2FF000C11CF101C11DF102C11EF1C0
:105DF00003C11FF1120E64EC0BF0E8CF04F1130E97
:105E000064EC0BF0E8CF05F1140E64EC0BF0E8CF76
:105E100006F1150E64EC0BF0E8CF07F10D0E006FE4
:105E2000000E016F000E026F000E036F78EC2FF072
:105E3000180E046F000E056F000E066F000E076F40
:105E400098EC2FF01CC104F11DC105F11EC106F133
:105E50001FC107F16CEC2FF06A0E046F2A0E056F5C
:105E6000000E066F000E076F67EC2FF01200BF0EDA
:105E7000FA6E200E3A6F396BD8900037013702372F
:105E80000337D8B048EF2FF03A2F3DEF2FF0390706
:105E90003A070353D8B412000331070B80093F6F50
:105EA00003390F0B010F396F80EC5FF0406F39053C
:105EB00080EC5FF0405D405F396B3F33D8B03927ED
:105EC00039333FA95DEF2FF040513927120001010E
:105ED00087EC30F0D8B01200010103510719346F7C
:105EE0004AEC30F0D8900751031934AF800F1200FC
:105EF0000101346B6EEC30F0D8A084EC30F0D8B0F7
:105F0000120059EC30F062EC30F01F0E366F9AEC54
:105F100030F00B35D8B04AEC30F0D8A00335D8B00B
:105F20001200362F87EF2FF034B171EC30F01200F1
:105F30000101346B04510511061107110008D8A0A6
:105F40006EEC30F0D8A084EC30F0D8B01200086BC2
:105F5000096B0A6B0B6B9AEC30F01F0E366F9AECE4
:105F600030F007510B5DD8A4C2EF2FF006510A5D47
:105F7000D8A4C2EF2FF00551095DD8A4C2EF2FF0CD
:105F80000451085DD8A0D5EF2FF00451085F0551EA
:105F9000D8A0053D095F0651D8A0063D0A5F07510C
:105FA000D8A0073D0B5FD8900081362FAFEF2FF0C0
:105FB00034B171EC30F0346B6EEC30F0D8909EEC74
:105FC00030F007510B5DD8A4F2EF2FF006510A5DB7
:105FD000D8A4F2EF2FF00551095DD8A4F2EF2FF00D
:105FE0000451085DD8A001EF30F0003F01EF30F020
:105FF000013F01EF30F0023F01EF30F0032BD8B446
:10600000120034B171EC30F012000101346B6EEC0F
:1060100030F0D8B01200A3EC30F0200E366F00370D
:1060200001370237033711EE33F00A0E376FE736C8
:106030000A0EE75CD8B0E76EE552372F17EF30F065
:10604000362F0FEF30F034B12981D89012000101C2
:106050000A0E346F200E366F11EE29F03451376F6F
:106060000A0ED890E652D8B0E726E732372F32EF43
:1060700030F00333023301330033362F2CEF30F08E
:10608000E750FF0FD8A00335D8B0120029B171EC4A
:1060900030F01200045100270551D8B0053D01270A
:1060A0000651D8B0063D02270751D8B0073D032757
:1060B00012000051086F0151096F02510A6F03511C
:1060C0000B6F12000101006B016B026B036B12007E
:1060D0000101046B056B066B076B12000335D8A03A
:1060E00012000351800B001F011F021F031F003FFE
:1060F00081EF30F0013F81EF30F0023F81EF30F06F
:10610000032B342B032512000735D8A012000751AA
:10611000800B041F051F061F071F043F97EF30F079
:10612000053F97EF30F0063F97EF30F0072B342B09
:1061300007251200003701370237033708370937C0
:106140000A370B3712000101296B2A6B2B6B2C6B62
:106150002D6B2E6B2F6B306B316B326B336B1200F0
:1061600001012A510F0B2A6F2B510F0B2B6F2C5152
:106170000F0B2C6F2D510F0B2D6F2E510F0B2E6F00
:106180002F510F0B2F6F30510F0B306F31510F0B01
:10619000316F32510F0B326F33510F0B336F1200CF
:1061A00000C124F101C125F102C126F103C127F18B
:1061B00004C100F105C101F106C102F107C103F1FB
:1061C00024C104F125C105F126C106F127C107F15B
:1061D000120010A806D08994000EC76E220EC66E5B
:1061E00005D08984000EC76E220EC66E050EE82EFD
:1061F000FED7120010A802D0898401D08994050E20
:10620000E82EFED71200E9EC30F09E96C69E000EF6
:10621000C96EFF0E9EB602D0E82EFCD79E96C69E93
:10622000000EC96EFF0E9EB602D0E82EFCD7C9CF75
:10623000AFF59E96C69E000EC96EFF0E9EB602D0AA
:10624000E82EFCD7C9CFB0F59E96C69E000EC96E4B
:10625000FF0E9EB602D0E82EFCD7C9CFB1F59E96B0
:10626000C69E000EC96EFF0E9EB602D0E82EFCD769
:10627000C9CFB2F59E96C69E000EC96EFF0E9EB6A1
:1062800002D0E82EFCD7C9CFB3F59E96C69E000E6D
:10629000C96EFF0E9EB602D0E82EFCD7C9CFB4F56A
:1062A0009E96C69E000EC96EFF0E9EB602D0E82EC8
:1062B000FCD7C9CFB5F5FAEC30F01200E9EC30F0BC
:1062C0009E96C69E800EC96EFF0E9EB602D0E82E28
:1062D000FCD79E96C69EAFC5C9FFFF0E9EB602D0E4
:1062E000E82EFCD79E96C69EB0C5C9FFFF0E9EB68F
:1062F00002D0E82EFCD79E96C69EB1C5C9FFFF0E00
:106300009EB602D0E82EFCD79E96C69EB2C5C9FFA7
:10631000FF0E9EB602D0E82EFCD79E96C69EB3C551
:10632000C9FFFF0E9EB602D0E82EFCD79E96C69EF1
:10633000B4C5C9FFFF0E9EB602D0E82EFCD79E96CC
:10634000C69EB5C5C9FFFF0E9EB602D0E82EFCD78B
:10635000FAEC30F01200E9EC30F09E96C69E070E83
:10636000C96EFF0E9EB602D0E82EFCD79E96C69E42
:10637000000EC96EFF0E9EB602D0E82EFCD7C9CF24
:10638000AFF59E96C69E000EC96EFF0E9EB602D059
:10639000E82EFCD7C9CFB0F59E96C69E000EC96EFA
:1063A000FF0E9EB602D0E82EFCD7C9CFB1F59E965F
:1063B000C69E000EC96EFF0E9EB602D0E82EFCD718
:1063C000C9CFB2F5FAEC30F0E9EC30F09E96C69EFB
:1063D00025C0C9FFFF0E9EB602D0E82EFCD79E96C0
:1063E000C69E000EC96EFF0E9EB602D0E82EFCD7E8
:1063F000C9CFB6F5FAEC30F01200E9EC30F09E9619
:10640000C69E870EC96EFF0E9EB602D0E82EFCD740
:106410009E96C69EAFC5C9FFFF0E9EB602D0E82E5F
:10642000FCD79E96C69EB0C5C9FFFF0E9EB602D091
:10643000E82EFCD79E96C69EB1C5C9FFFF0E9EB63C
:1064400002D0E82EFCD79E96C69EB2C5C9FFFF0EAD
:106450009EB602D0E82EFCD7FAEC30F0E9EC30F032
:106460009E96C69E26C0C9FFFF0E9EB602D0E82E9D
:10647000FCD79E96C69EB6C5C9FFFF0E9EB602D03B
:10648000E82EFCD7FAEC30F01200E9EC30F09E96E2
:10649000C69E870EC96EFF0E9EB602D0E82EFCD7B0
:1064A0009E96C69E000EC96EFF0E9EB602D0E82EC6
:1064B000FCD79E96C69E800EC96EFF0E9EB602D079
:1064C000E82EFCD79E96C69E800EC96EFF0E9EB625
:1064D00002D0E82EFCD79E96C69E800EC96EFF0E97
:1064E0009EB602D0E82EFCD7FAEC30F01200E9ECB0
:1064F00030F09E96C69E870EC96EFF0E9EB602D0E5
:10650000E82EFCD79E96C69E000EC96EFF0E9EB664
:1065100002D0E82EFCD79E96C69E000EC96EFF0ED6
:106520009EB602D0E82EFCD79E96C69E800EC96EFF
:10653000FF0E9EB602D0E82EFCD79E96C69E800E19
:10654000C96EFF0E9EB602D0E82EFCD7FAEC30F0F2
:10655000120010A817D0E9EC30F09E96C69E8F0E60
:10656000C96EFF0E9EB602D0E82EFCD79E96C69E40
:10657000000EC96EFF0E9EB602D0E82EFCD7FAECD4
:1065800030F01200ABEC31F0120010A82DD0E9EC85
:1065900030F09E96C69E26C0C9FFFF0E9EB602D062
:1065A000E82EFCD79E96C69E450EC96EFF0E9EB67F
:1065B00002D0E82EFCD7FAEC30F0E9EC30F09E96F1
:1065C000C69E8F0EC96EFF0E9EB602D0E82EFCD777
:1065D0009E96C69E000EC96EFF0E9EB602D0E82E95
:1065E000FCD7FAEC30F01200E9EC30F09E96C69E33
:1065F00026C0C9FFFF0E9EB602D0E82EFCD79E969D
:10660000C69E010EC96EFF0E9EB602D0E82EFCD7C4
:10661000FAEC30F0E9EC30F09E96C69E910EC96E11
:10662000FF0E9EB602D0E82EFCD79E96C69EA50E03
:10663000C96EFF0E9EB602D0E82EFCD7FAEC30F001
:106640001200E9EC30F09E96C69E26C0C9FFFF0EF0
:106650009EB602D0E82EFCD79E96C69E810EC96ECD
:10666000FF0E9EB602D0E82EFCD7FAEC30F01200F6
:10667000E9EC30F09E96C69E26C0C9FFFF0E9EB67E
:1066800002D0E82EFCD79E96C69E010EC96EFF0E64
:106690009EB602D0E82EFCD7FAEC30F01200E9ECFE
:1066A00030F09E96C69E910EC96EFF0E9EB602D029
:1066B000E82EFCD79E96C69EA50EC96EFF0E9EB60E
:1066C00002D0E82EFCD7FAEC30F01200E9EC30F002
:1066D0009E96C69E910EC96EFF0E9EB602D0E82E03
:1066E000FCD79E96C69E000EC96EFF0E9EB602D0C7
:1066F000E82EFCD7FAEC30F012000501256B266B72
:10670000276B286B899A400EC76E200EC66E9E9628
:10671000C69E030EC96EFF0E9EB602D0E82EFCD7B1
:106720009E96C69E27C5C9FFFF0E9EB602D0E82ED4
:10673000FCD79E96C69E26C5C9FFFF0E9EB602D008
:10674000E82EFCD79E96C69E25C5C9FFFF0E9EB6B5
:1067500002D0E82EFCD79E96C69EC952FF0E9EB66A
:1067600002D0E82EFCD7898A0F01C950FF0A01E147
:10677000120005012E51130A05E005012E51170ADA
:106780000CE012000501F00E256FFF0E266F0F0EB4
:10679000276F000E286FD6EF33F00501F00E256F3E
:1067A000FF0E266FFF0E276F000E286F899A400E8E
:1067B000C76E200EC66E9E96C69E030EC96EFF0E55
:1067C0009EB602D0E82EFCD79E96C69E27C5C9FF6E
:1067D000FF0E9EB602D0E82EFCD79E96C69E26C51A
:1067E000C9FFFF0E9EB602D0E82EFCD79E96C69E2D
:1067F00025C5C9FFFF0E9EB602D0E82EFCD79E9697
:10680000C69EC952FF0E9EB602D0E82EFCD7898ADA
:106810000F01C950FF0A1DE005012E51130A05E0C2
:1068200005012E51170A0BE012000501000E256F1D
:10683000000E266F100E276F000E286F1200050144
:10684000000E256F000E266F000E276F010E286FB9
:1068500012000501256B266B276B286B05012E5155
:10686000130A05E005012E51170A0CE0120005017C
:10687000000E216F000E226F080E236F000E246F92
:106880004BEF34F00501000E216F000E226F800ED9
:10689000236F000E246F21C500F122C501F123C52D
:1068A00002F124C503F125C504F126C505F127C56C
:1068B00006F128C507F1B8EC2DF000C125F501C19E
:1068C00026F502C127F503C128F5899A400EC76E47
:1068D000200EC66E9E96C69E030EC96EFF0E9EB615
:1068E00002D0E82EFCD79E96C69E27C5C9FFFF0E94
:1068F0009EB602D0E82EFCD79E96C69E26C5C9FF3E
:10690000FF0E9EB602D0E82EFCD79E96C69E25C5E9
:10691000C9FFFF0E9EB602D0E82EFCD79E96C69EFB
:10692000C952FF0E9EB602D0E82EFCD7898AC95004
:10693000FF0A08E104C125F505C126F506C127F5C2
:1069400007C128F5D890050124332333223321339E
:106950002151F00B216F05012167B6EF34F022675A
:10696000B6EF34F02367B6EF34F024674BEF34F022
:106970000501100E2527E86A2623E86A2723E86A1E
:1069800028231200E86A05012E51130A06E00501CA
:106990002E51170A0BE0020E120005012851000AC1
:1069A00003E12751F00B07E0010E12000501285109
:1069B000000A01E0010E120029C500F12AC501F10B
:1069C0002BC502F12CC503F125C504F126C505F13F
:1069D00027C506F128C507F167EC2FF003BF1200A9
:1069E000C2EC34F0D8A454EF35F0899A400EC76E4B
:1069F000200EC66E9E96C69E060EC96EFF0E9EB6F1
:106A000002D0E82EFCD7898A899A9E96C69E020EED
:106A1000C96EFF0E9EB602D0E82EFCD79E96C69E8B
:106A200027C5C9FFFF0E9EB602D0E82EFCD79E9662
:106A3000C69E26C5C9FFFF0E9EB602D0E82EFCD723
:106A40009E96C69E25C5C9FFFF0E9EB602D0E82EB3
:106A5000FCD79E96C69E000EC96EFF0E9EB602D053
:106A6000E82EFCD7898A899A9E96C69E050EC96E25
:106A7000FF0E9EB602D0E82EFCD79E96C69EC95247
:106A8000FF0E9EB602D0E82EFCD7C9B03DEF35F020
:106A9000898A0501100E2527E86A2623E86A27233C
:106AA000E86A2823DCEF34F01200899A400EC76EA2
:106AB000200EC66E9E96C69E060EC96EFF0E9EB630
:106AC00002D0E82EFCD7898A899A9E96C69EC70E68
:106AD000C96EFF0E9EB602D0E82EFCD7898A05014A
:106AE000256B266B276B286B1200899A400EC76EA8
:106AF000200EC66E9E96C69E050EC96EFF0E9EB6F1
:106B000002D0E82EFCD79E96C69EC952FF0E9EB6B6
:106B100002D0E82EFCD7C9CF37F5898A1200899AAE
:106B2000400EC76E200EC66E9E96C69EB90EC96EEA
:106B3000FF0E9EB602D0E82EFCD7898A1200899AF1
:106B4000400EC76E200EC66E9E96C69EAB0EC96ED8
:106B5000FF0E9EB602D0E82EFCD7898AFF0EE82EE3
:106B6000FED71200C2EC34F0D8A41200899A400E6D
:106B7000C76E200EC66E9E96C69E030EC96EFF0E91
:106B80009EB602D0E82EFCD79E96C69E27C5C9FFAA
:106B9000FF0E9EB602D0E82EFCD79E96C69E26C556
:106BA000C9FFFF0E9EB602D0E82EFCD79E96C69E69
:106BB00025C5C9FFFF0E9EB602D0E82EFCD79E96D3
:106BC000C69EC952FF0E9EB602D0E82EFCD7898A17
:106BD0000F01C950FF0AD8A40AEF37F00501FE0ED5
:106BE000376F15A63799158603EC31F0AFC538F528
:106BF000B0C539F5B1C53AF5B2C53BF5B3C53CF5FD
:106C0000B4C53DF5B5C53EF50784BAC166F1BBC153
:106C100067F1BCC168F1BDC169F14BC14FF14CC115
:106C200050F14DC151F14EC152F157C159F158C106
:106C30005AF100011650010AD8B42DEF36F00001C8
:106C40001650020AD8B443EF36F000011650040A79
:106C5000D8B459EF36F00AEF37F08BA0379B61ECD0
:106C600022F000C1DAF101C1DBF102C1DCF103C1A4
:106C7000DDF100C13FF501C140F502C141F503C19D
:106C800042F578EF36F061EC22F000C1DAF101C193
:106C9000DBF102C1DCF103C1DDF15EEC23F000C1E8
:106CA00047F501C148F502C149F503C14AF50AEFAC
:106CB00037F0379BDAC13FF5DBC140F5DCC141F568
:106CC000DDC142F561EC22F000C14BF501C14CF58C
:106CD00002C14DF503C14EF55EEC23F000C14FF546
:106CE00001C150F502C151F503C152F578EF36F0FC
:106CF0000501616783EF36F0626783EF36F0636703
:106D000083EF36F0646787EF36F09CEF36F0DAC138
:106D100000F1DBC101F1DCC102F1DDC103F161C5AC
:106D200004F162C505F163C506F164C507F167ECBE
:106D30002FF003BF0AEF37F059C143F55AC144F5AC
:106D4000B9C545F50501110E326F899A400EC76E1F
:106D5000200EC66E9E96C69E060EC96EFF0E9EB68D
:106D600002D0E82EFCD7898A899A9E96C69E020E8A
:106D7000C96EFF0E9EB602D0E82EFCD79E96C69E28
:106D800027C5C9FFFF0E9EB602D0E82EFCD79E96FF
:106D9000C69E26C5C9FFFF0E9EB602D0E82EFCD7C0
:106DA0009E96C69E25C5C9FFFF0E9EB602D0E82E50
:106DB000FCD725EE37F0322F02D0EAEF36F09E9660
:106DC000C69EDECFC9FFFF0E9EB602D0E82EFCD7CE
:106DD000DBEF36F0898A899A9E96C69E050EC96EAB
:106DE000FF0E9EB602D0E82EFCD79E96C69EC952D4
:106DF000FF0E9EB602D0E82EFCD7C9B0F5EF36F0F4
:106E0000898A0501100E2527E86A2623E86A2723C8
:106E1000E86A282315900794120021C500F122C5C5
:106E200001F123C502F124C503F1899A400EC76E12
:106E3000200EC66E9E96C69E0B0EC96EFF0E9EB6A7
:106E400002D0E82EFCD79E96C69E02C1C9FFFF0E57
:106E50009EB602D0E82EFCD79E96C69E01C1C9FF01
:106E6000FF0E9EB602D0E82EFCD79E96C69E00C1AD
:106E7000C9FFFF0E9EB602D0E82EFCD79E96C69E96
:106E8000C952FF0E9EB602D0E82EFCD725EE37F091
:106E90000501100E326F9E96C69EC952FF0E9EB619
:106EA00002D0E82EFCD7C9CFDEFF322F4BEF37F0F0
:106EB000898A1200899A400EC76E200EC66E9E9671
:106EC000C69E900EC96EFF0E9EB602D0E82EFCD76D
:106ED0009E96C69E000EC96EFF0E9EB602D0E82E8C
:106EE000FCD79E96C69E000EC96EFF0E9EB602D0BF
:106EF000E82EFCD79E96C69E000EC96EFF0E9EB66B
:106F000002D0E82EFCD79E96C69EC952FF0E9EB6B2
:106F100002D0E82EFCD7C9CF2DF59E96C69EC95249
:106F2000FF0E9EB602D0E82EFCD7C9CF2EF5898A77
:106F3000120003EC31F005012F51020A16E00501A1
:106F40002F51030A19E005012F51040A24E005011D
:106F50002F51050A2BE005012F51060A39E00501E2
:106F60002F51070A3FE0FAEF37F0602FF8EF37F0C4
:106F70005FC560F5FAEF37F0B0C500F101010F0E03
:106F8000001701010051000A35E001010051050A16
:106F900031E0F8EF37F0B0C500F101010F0E001736
:106FA00001010051000A26E0F8EF37F00501B05169
:106FB000000A20E00501B051150A1CE00501B0519E
:106FC000300A18E00501B051450A14E0F8EF37F037
:106FD0000501B051000A0EE00501B051300A0AE087
:106FE000F8EF37F00501B051000A04E0F8EF37F090
:106FF00015901200158012008B9033EC2EF0B9C55D
:10700000E8FFD70802E333EC2EF0B9C5E8FFC80863
:1070100002E333EC2EF0B9C5E8FFB90802E333EC24
:107020002EF0B9C5E8FFAA0802E333EC2EF0B9C58B
:10703000E8FF9B0802E333EC2EF08FEC35F0F29C76
:10704000F29E8B94C69AC2909482948C720ED36EE8
:10705000D3A4FED789968A909390F29AF2949D9049
:107060009E909D929E92F298F292A9EC32F0FF0EC1
:10707000E8CF00F0E82EFED7002EFCD7F290F28683
:10708000815081A846EF38F0F29E0300700ED36E57
:10709000F296F2901584038054EC2EF09AEF0BF0E8
:10BF0000E844F926000C160C2B0C3F0C520C640C68
:10BF1000760C860C960CA50CB30CC10CCF0CDC0C6B
:06BF2000E80CF40C000C1B
:0200000400F00A
:0100C800FE39
:00000001FF
